:0200000480007A
:10000000B72F0000938F0F8073900F306F00400365
:100010001300000013000000130000001300000094
:100020001300000013000000130000001300000084
:100030001300000013000000130000001300000074
:100040009702000093824211739052309300000097
:10005000130100009301000013020000930200004E
:100060001303000093030000130400009304000036
:10007000130500009305000013060000930600001E
:100080001307000093070000130800009308000006
:100090001309000093090000130A0000930A0000EE
:1000A000130B0000930B0000130C0000930C0000D6
:1000B000130D0000930D0000130E0000930E0000BE
:1000C000130F0000930F000097110200938181B17C
:1000D0001705020013050533979503009385C5673F
:1000E00013060000EF00001A170502001305C52EC5
:1000F000970502009385C52E13060000EF008018B7
:1001000017A503001305856597B503009385C5649E
:1001100037B6ABAB1306B6BAEF00C01617B1030083
:100120001301C163EF7080759392120093D2120095
:100130009382D2FF638A02008322010013014100EF
:100140006F0000177300203083220100130141006B
:10015000730020301301C1FF23205100F32220340B
:10016000E3C402FC8322010013014100130141F8A2
:1001700023221100232421002326310023284100BB
:10018000232A5100232C6100232E71002320810299
:10019000232291022324A1022326B1022328C10293
:1001A000232AD102232CE102232EF1022320010570
:1001B0002322110523242105232631052328410567
:1001C000232A5105232C6105232E71052320810745
:1001D000232291072324A1072326B1072328C1073F
:1001E000232AD107232CE107232EF107732520347E
:1001F000F3251034130601006F000000731015344E
:1002000083204100032181008321C10003220101D9
:1002100083224101032381018323C10103240102BD
:1002200083244102032581028325C10203260103A1
:1002300083264103032781038327C1030328010485
:1002400083284104032981048329C104032A010569
:10025000832A4105032B8105832BC105032C01064D
:10026000832C4106032D8106832DC106032E010731
:10027000832E4107032F8107832FC1071301C10775
:10028000730020302320C5006376B50013054500B8
:100290006FF05FFF678000000000000000000000BA
:1002A000000000000000000000000000000000004E
:1002B000130101F8232011002322210023243100FF
:1002C0002326410023285100232A6100232C71009A
:1002D000232E8100232091022322A1022324B10294
:1002E0002326C1022328D102232AE102232CF10272
:1002F000232E010323201105232221052324310568
:100300002326410523285105232A6105232C710545
:10031000232E8105232091072322A1072324B1073F
:100320002326C1072328D107232AE107232CF1071D
:100330009702020083A2420A23A02200F322103473
:10034000232E5106EF008046170102000321C10849
:10035000032101008322C10773901234B7220000E9
:100360009382028873A00230832001000322C1001F
:100370008322010103234101832381010324C1015D
:100380008324010203254102832581020326C10241
:100390008326010303274103832781030328C10325
:1003A000832801040329410483298104032AC10409
:1003B000832A0105032B4105832B8105032CC105ED
:1003C000832C0106032D4106832D8106032EC106D1
:1003D000832E0107032F4107832F81071301010893
:1003E00073002030970202009382C20123A0120002
:1003F00023A2220023A4320023A6420023A85200F5
:1004000023AA620023AC720023AE820023A09202D2
:1004100023A2A20223A4B20223A6C20223A8D202CC
:1004200023AAE20223ACF20223AE020323A01205A8
:1004300023A2220523A4320523A6420523A85205A0
:1004400023AA620523AC720523AE820523A092077E
:1004500023A2A20723A4B20723A6C20723A8D20778
:1004600023AAE20723ACF207EF704027170102002E
:10047000032181F6032101008322C1077390123406
:10048000B72200009382028873A00230832001000B
:100490000322C1008322010103234101832381013F
:1004A0000324C10183240102032541028325810223
:1004B0000326C10283260103032741038327810307
:1004C0000328C103832801040329410483298104EB
:1004D000032AC104832A0105032B4105832B8105CF
:1004E000032CC105832C0106032D4106832D8106B3
:1004F000032EC106832E0107032F4107832F810797
:10050000130101087300203097020200938282EFEA
:1005100083A0020003A1420083A1820003A2C200C3
:1005200083A2020103A3420183A3820103A4C201A7
:1005300083A4020203A5420283A5820203A6C2028B
:1005400083A6020303A7420383A7820303A8C2036F
:1005500083A8020403A9420483A9820403AAC20453
:1005600083AA020503AB420583AB820503ACC20537
:1005700083AC020603AD420683AD820603AEC2061B
:1005800083AE020703AFC20983AF82076780000012
:1005900073700430130101F823201100232221007D
:1005A000232431002326410023285100232A6100FF
:1005B000232C7100232E8100232091022322A102EB
:1005C0002324B1022326C1022328D102232AE102D7
:1005D000232CF102232E01032320110523222105C0
:1005E000232431052326410523285105232A6105AB
:1005F000232C7105232E8105232091072322A10797
:100600002324B1072326C1072328D107232AE10782
:10061000232CF1079702020083A202DC23A0220010
:10062000232E1106EF30000D170102000321C1DA5D
:10063000032101008322C10773901234B722000006
:100640009382028873A00230832001000322C1003C
:100650008322010103234101832381010324C1017A
:100660008324010203254102832581020326C1025E
:100670008326010303274103832781030328C10342
:10068000832801040329410483298104032AC10426
:10069000832A0105032B4105832B8105032CC1050A
:1006A000832C0106032D4106832D8106032EC106EE
:1006B000832E0107032F4107832F810713010108B0
:1006C00073002030970702009387C7D103A7070064
:1006D0009307F0FF6306F700737004306F000000AB
:1006E000737004306F000000130101FF2326A10086
:1006F0008327C100739047301300000013010101EC
:1007000067800000130101FFF32740302326F1002A
:1007100073F043308327C1001385070013010101E3
:1007200067800000130101FF2326A1002324B100EC
:100730002322C1008327C1009387C7FF2326F1002E
:10074000032781008327C10023A0E7008327C1007E
:10075000938787FA2326F100032741008327C100EE
:1007600023A0E7008327C100938787FE2326F1009B
:1007700093870100138707008327C10023A0E700A8
:100780008327C100938747FF2326F1001707000046
:10079000130787F38327C10023A0E7008327C10045
:1007A000138507001301010167800000130101FF99
:1007B00023261100EF601068EF20504A93070500D0
:1007C00063840700EF201073130000008320C10032
:1007D0001301010167800000130101FF2326A1001E
:1007E0008327C100138787008327C10023A2E70066
:1007F0008327C1001307F0FF23A4E7008327C1006C
:10080000138787008327C10023A6E7008327C10041
:10081000138787008327C10023A8E7008327C1002F
:1008200023A00700130000001301010167800000EE
:10083000130101FF2326A1008327C10023A807007D
:10084000130000001301010167800000130101FE85
:100850002326A1002324B1008327C10083A74700DA
:10086000232EF100832781000327C10123A2E70083
:100870008327C10103A787008327810023A4E70002
:100880008327C10183A787000327810023A2E700F4
:100890008327C1010327810023A4E7008327810068
:1008A0000327C10023A8E7008327C10083A707000F
:1008B000138717008327C10023A0E700130000005F
:1008C0001301010267800000130101FE2326A1002D
:1008D0002324B1008327810083A70700232CF10084
:1008E000032781019307F0FF631AF7008327C100F4
:1008F00083A70701232EF1006F0040038327C10067
:1009000093878700232EF1006F0000018327C10128
:1009100083A74700232EF1008327C10183A7470047
:1009200083A7070003278101E372F7FE8327C10134
:1009300003A747008327810023A2E70083278100C4
:1009400083A747000327810023A4E70083278100B2
:100950000327C10123A4E7008327C10103278100E6
:1009600023A2E700832781000327C10023A8E70013
:100970008327C10083A70700138717008327C100BF
:1009800023A0E700130000001301010267800000AC
:10099000130101FE2326A1008327C10083A70701BD
:1009A000232EF1008327C10083A747000327C1003E
:1009B0000327870023A4E7008327C10083A78700BC
:1009C0000327C1000327470023A2E7008327C101B3
:1009D00083A747000327C100631AF7008327C100DC
:1009E00003A787008327C10123A2E7008327C10053
:1009F00023A807008327C10183A707001387F7FFF8
:100A00008327C10123A0E7008327C10183A7070033
:100A1000138507001301010267800000130101FD27
:100A200023261102232481022326A1002324B100BE
:100A30008327C100232EF1008327C101639607009D
:100A4000737004306F000000EF3050758327C101D0
:100A500003A407008327C10103A7C7038327C1019C
:100A600083A707049385070013050700EF80006341
:100A7000930705003307F4008327C10123A2E70091
:100A80008327C10123AC07028327C10103A7070005
:100A90008327C10123A4E7008327C10103A4070022
:100AA0008327C10183A7C7031387F7FF8327C101EA
:100AB00083A707049385070013050700EF80005EF6
:100AC000930705003307F4008327C10123A6E7003D
:100AD0008327C1011307F0FF23A2E7048327C10185
:100AE0001307F0FF23A4E70483278100639A07021A
:100AF0008327C10183A70701638407048327C101FA
:100B00009387070113850700EF3080001307050066
:100B1000930710006316F702EFF09FA76F004002E3
:100B20008327C1019387070113850700EFF0DFCA10
:100B30008327C1019387470213850700EFF0DFC9C0
:100B4000EF30D06993071000138507008320C1029E
:100B5000032481021301010367800000130101FDDA
:100B6000232611022326A1002324B10093070600A7
:100B7000A303F100232C01008327C1006396070023
:100B8000737004306F0000008327810063960700B4
:100B9000232E01006F00C001832581000325C100C1
:100BA000EF80C04F9307050093871700232EF100B5
:100BB0008327C1019387870513850700EF505022D3
:100BC000232AA1008327410163860706832781002A
:100BD000639A0700832741010327410123A0E7000F
:100BE0006F00400183274101138787058327410157
:100BF00023A0E700832741010327C10023AEE702BA
:100C0000832741010327810023A0E70493051000F7
:100C100003254101EFF09FE0832741010347710065
:100C20002388E7048327410123AA0704832741017E
:100C3000232CF10083278101639607007370043031
:100C40006F00000083278101138507008320C10204
:100C50001301010367800000130101FD2326110227
:100C600093070500A307F10013058005EF50501707
:100C7000232EA1008327C1016380070A8327C101B6
:100C800023A207008327C10123A007008327C101F6
:100C900023A407008327C10123A607008327C101DE
:100CA00023AC07028327C1011307100023AEE7021C
:100CB0008327C10123A007048327C1011307F0FF85
:100CC00023A2E7048327C1011307F0FF23A4E7044D
:100CD0008327C1010347F1002388E7048327C1016B
:100CE00023AA07048327C1019387070113850700FF
:100CF000EFF09FAE8327C10193874702138507005A
:100D0000EFF09FAD9306000013060000930500006E
:100D10000325C101EF00001E8327C10113850700D1
:100D20008320C1021301010367800000130101FD4C
:100D300023261102232481022326A1008327C10038
:100D4000232CF10083278101639607007370043020
:100D50006F0000008327810103A44700EF30501388
:100D6000930705006312F4048327810183A7C7005A
:100D70001387F7FF8327810123A6E70083278101DB
:100D800083A7C700639C07009306000013060000BA
:100D90009305000003258101EF00C01593071000A3
:100DA000232EF1006F008000232E01008327C10154
:100DB000138507008320C10203248102130101036C
:100DC00067800000130101FD232611022324810204
:100DD0002326A1002324B1008327C100232CF10086
:100DE0008327810163960700737004306F00000051
:100DF0008327810103A44700EF3090099307050082
:100E00006312F4028327810183A7C70013871700A9
:100E10008327810123A6E70093071000232EF1000A
:100E20006F00C003930600000326810093050000B5
:100E300003258101EF000063232EA1000327C101D8
:100E400093071000631CF7008327810183A7C70065
:100E5000138717008327810123A6E7008327C10199
:100E6000138507008320C1020324810213010103BB
:100E700067800000130101FD232611022326A10033
:100E80002324B1008327C1006396070073700430E8
:100E90006F000000032781008327C10063F6E7008D
:100EA000737004306F0000001306200093050000EB
:100EB0000325C100EFF09FCA232EA1008327C101A3
:100EC000638807008327C1010327810023ACE70261
:100ED0008327C10163960700737004306F00000020
:100EE0008327C101138507008320C1021301010379
:100EF00067800000130101FC232E11022326A100AC
:100F00002324B1002322C1002320D1002326010283
:100F10008327C1002324F1028327810263960700FF
:100F2000737004306F00000083278100639807000E
:100F30008327810283A707046396070093071000A5
:100F40006F00800093070000639607007370043001
:100F50006F0000000327010093072000631AF700C9
:100F60008327810203A7C703930710006316F700C6
:100F7000930710006F00800093070000639607003E
:100F8000737004306F000000EF30C07293070500EB
:100F900063960700832741006396070093071000BC
:100FA0006F008000930700006396070073700430A1
:100FB0006F000000EF30901E8327810203A7870394
:100FC0008327810283A7C7036368F7000327010013
:100FD000930720006316F70803260100832581008C
:100FE00003258102EF0050262322A10283278102DC
:100FF00083A7470563820702832501000325810239
:10100000EF10401A13070500930710006314F7044C
:10101000EFF00FD86F0000048327810283A74702F7
:1010200063840702832781029387470213850700A1
:10103000EF20102E1307050093071000631CF70024
:10104000EFF00FD56F000001832741026384070092
:10105000EFF00FD4EF309018930710006F00400F9F
:101060008327410063980700EF3050179307000073
:101070006F00000E8327C102639C07009307C10124
:1010800013850700EF20D04D930710002326F102AF
:10109000EF30D014EF10507AEF30501083278102D8
:1010A00003A747049307F0FF6316F7008327810225
:1010B00023A207048327810203A787049307F0FF75
:1010C0006316F7008327810223A40704EF30101171
:1010D000130741009307C10193050700138507001B
:1010E000EF20D04C93070500639C07040325810281
:1010F000EF00905093070500638C0702832781025D
:101100009387070103274100930507001385070014
:10111000EF20807A03258102EF001034EF10107465
:1011200093070500E39807E8EFF08FC66FF09FE89C
:1011300003258102EF005032EF1050726FF09FE7ED
:1011400003258102EF005031EF105071930700002A
:10115000138507008320C103130101046780000089
:10116000130101FD232611022326A1002324B1002F
:101170002322C1002320D1008327C100232CF100AA
:101180008327810163960700737004306F000000AD
:1011900083278100639807008327810183A70704C1
:1011A00063960700930710006F008000930700000C
:1011B00063960700737004306F000000032701007E
:1011C00093072000631AF7008327810103A7C70351
:1011D000930710006316F700930710006F0080005C
:1011E0009307000063960700737004306F000000DF
:1011F000EFF04FD193070500232AF10083278101E7
:1012000003A787038327810183A7C7036368F700C8
:101210000327010093072000631EF70A032601003D
:101220008325810003258101EF00100283278101BE
:1012300003A787049307F0FF631EF7068327810146
:1012400083A74705638A07028325010003258101DF
:10125000EF00507513070500930710006316F7069B
:10126000832741006382070683274100130710008C
:1012700023A0E7006F0040058327810183A7470271
:10128000638407048327810193874702138507003E
:10129000EF201008930705006388070283274100A9
:1012A00063840702832741001307100023A0E7008F
:1012B0006F0080018327810183A7870413871700AC
:1012C0008327810123A4E70493071000232EF10054
:1012D0006F008000232E0100832741011385070042
:1012E000EFF08FC08327C101138507008320C1025F
:1012F0001301010367800000130101FD2326110281
:101300002326A1002324B1008327C100232CF10050
:101310008327810163960700737004306F0000001B
:101320008327810183A70704638607007370043055
:101330006F0000008327810183A7070063980700DF
:101340008327810183A74700639607009307100056
:101350006F008000930700006396070073700430ED
:101360006F000000EFF00FBA93070500232AF10089
:101370008327810103A787038327810183A7C703ED
:101380006370F70C8327810183A7870313871700F6
:101390008327810123ACE7028327810103A7870408
:1013A0009307F0FF631EF7068327810183A7470594
:1013B000638A07029305000003258101EF00905E18
:1013C00013070500930710006316F70683278100B3
:1013D00063820706832781001307100023A0E7001C
:1013E0006F0040058327810183A7470263840704B8
:1013F000832781019387470213850700EF204071FF
:10140000930705006388070283278100638407022E
:10141000832781001307100023A0E7006F008001DD
:101420008327810183A787041387170083278101FE
:1014300023A4E70493071000232EF1006F0080001F
:10144000232E01008327410113850700EFF0CFA968
:101450008327C101138507008320C1021301010303
:1014600067800000130101FC232E11022326A10036
:101470002324B1002322C1002320D100232601020E
:101480008327C1002324F10283278102639607008A
:10149000737004306F000000832781006398070099
:1014A0008327810283A70704639607009307100030
:1014B0006F0080009307000063960700737004308C
:1014C0006F000000EF30001F9307050063960700D0
:1014D0008327410063960700930710006F00800088
:1014E0009307000063960700737004306F000000DC
:1014F000EF30C04A8327810283A787036382070CEA
:101500008327810283A7C7002322F102832581005C
:1015100003258102EF00806B832701006392070699
:101520008327810283A787031387F7FF832781021D
:1015300023ACE7028327810283A70700639A070091
:10154000EF308054130705008327810223A2E700B0
:101550008327810283A70701638E07048327810203
:101560009387070113850700EF20805A13070500B2
:10157000930710006310F704EFF08F816F00800372
:10158000832781020327410223A6E70083278102E4
:1015900083A747026380070283278102938747025C
:1015A00013850700EF20C0569307050063840700EA
:1015B000EFE01FFEEF308042930710006F008011B4
:1015C0008327410063980700EF30404193070000F4
:1015D0006F0040108327C102639C07009307C1017D
:1015E00013850700EF20C077930710002326F10230
:1015F000EF30C03EEF105024EF30403A8327810295
:1016000003A747049307F0FF6316F70083278102BF
:1016100023A207048327810203A787049307F0FF0F
:101620006316F7008327810223A40704EF30003BF1
:10163000130741009307C1019305070013850700B5
:10164000EF20C07693070500639E070603258102FD
:10165000EF00007293070500638E07048327810261
:1016600083A70700639E0700EF3040338327810282
:1016700083A7470013850700EF30C008EF3000361E
:1016800083278102938747020327410093050700C0
:1016900013850700EF20402203258102EF00C05B85
:1016A000EF10D01B93070500E39407E4EFE05FEE33
:1016B0006FF01FE403258102EF00005AEF10101AAB
:1016C0006FF01FE303258102EF000059EF1010199E
:1016D00093070000138507008320C1031301010451
:1016E00067800000130101FD232611022326A100BB
:1016F0002324B1002322C1008327C100232CF10041
:101700008327810163960700737004306F00000027
:1017100083278100639807008327810183A707043B
:1017200063960700930710006F0080009307000086
:1017300063960700737004306F000000EFE09FFCB9
:1017400093070500232AF1008327810183A78703DC
:10175000638807088325810003258101EF00004786
:101760008327810183A787031387F7FF83278101DD
:1017700023ACE7028327810103A747049307F0FF07
:101780006310F7048327810183A70701638407049B
:10179000832781019387070113850700EF204037D6
:1017A00093070500638807028327410063840702CB
:1017B000832741001307100023A0E7006F0080017A
:1017C0008327810183A7470413871700832781019B
:1017D00023A2E70493071000232EF1006F0080007E
:1017E000232E01008327410113850700EFE0DFEF7F
:1017F0008327C101138507008320C1021301010360
:1018000067800000130101FD232611022326A10099
:101810002324B1008327C100232CF10083278101F9
:1018200063960700737004306F0000008327810007
:10183000639807008327810183A707046396070045
:10184000930710006F008000930700006396070065
:10185000737004306F0000008327810183A70704A1
:1018600063960700737004306F000000EFE09FE99B
:1018700093070500232AF1008327810183A78703AB
:10188000638A07028327810183A7C7002328F10009
:101890008325810003258101EF00403383278101E7
:1018A0000327010123A6E70093071000232EF10070
:1018B0006F008000232E010083274101138507005C
:1018C000EFE09FE28327C101138507008320C10257
:1018D0001301010367800000130101FD232611029B
:1018E0002326A1008327C10063960700737004308C
:1018F0006F000000EF30800A8327C10083A78703B1
:10190000232EF100EF30800D8327C10113850700DE
:101910008320C1021301010367800000130101FD50
:10192000232611022326A1008327C100232EF100C4
:101930008327C10163960700737004306F000000B5
:10194000EF30C0058327C10103A7C7038327C10167
:1019500083A78703B307F740232CF100EF3000087B
:1019600083278101138507008320C102130101032E
:1019700067800000130101FE2326A1008327C10018
:1019800063960700737004306F0000008327C10066
:1019900083A78703232EF1008327C1011385070046
:1019A0001301010267800000130101FD23261102CB
:1019B0002326A1008327C100232EF1008327C10124
:1019C00063960700737004306F0000000325C101A7
:1019D000EF0000550325C101EF40506013000000E7
:1019E0008320C1021301010367800000130101FF7E
:1019F0002326A1008327C10083A7C70413850700FE
:101A00001301010167800000130101FF2326A100DB
:101A10002324B1008327C1000327810023A6E70404
:101A2000130000001301010167800000130101FF92
:101A30002326A1008327C10083C70705138507005C
:101A40001301010167800000130101FD232611022B
:101A50002326A1002324B1002322C100232E01004C
:101A60008327C10083A70704639807028327C10067
:101A700083A70700639807128327C10083A7470045
:101A800013850700EF20D05D232EA1008327C1001E
:101A900023A207006F00001183274100639407060B
:101AA0008327C10003A787008327C10083A70704FA
:101AB000138607008325810013050700EF40D068D7
:101AC0008327C10003A787008327C10083A70704DA
:101AD0003307F7008327C10023A4E7008327C10051
:101AE00003A787008327C10083A74700636CF70A19
:101AF0008327C10003A707008327C10023A4E700B1
:101B00006F00400A8327C10003A7C7008327C100D5
:101B100083A70704138607008325810013050700A8
:101B2000EF4090628327C10003A7C7008327C1004D
:101B300083A70704B307F0403307F7008327C100EA
:101B400023A6E7008327C10003A7C7008327C1009E
:101B500083A707006372F7028327C10003A747002A
:101B60008327C10083A70704B307F0403307F700BA
:101B70008327C10023A6E700032741009307200025
:101B80006312F7028327C10083A78703638C0700D2
:101B90008327C10083A787031387F7FF8327C1002B
:101BA00023ACE7028327C10083A7870313871700AD
:101BB0008327C10023ACE7028327C10113850700F7
:101BC0008320C1021301010367800000130101FE9D
:101BD000232E11002326A1002324B1008327C10056
:101BE00083A70704638207068327C10003A7C700F2
:101BF0008327C10083A707043307F7008327C100A9
:101C000023A6E7008327C10003A7C7008327C100DD
:101C100083A74700636AF7008327C10003A7070073
:101C20008327C10023A6E7008327C10003A7C700BD
:101C30008327C10083A707041386070093050700C5
:101C400003258100EF405050130000008320C101A4
:101C50001301010267800000130101FE232E110011
:101C60002326A100EF2090536F00C0068327C100F8
:101C700083A7470563820702930500000325C1007F
:101C8000EF0040521307050093071000631AF70294
:101C9000EF20C0216F00C0028327C10083A7470245
:101CA000638207048327C1009387470213850700D7
:101CB000EF1010669307050063840700EF20001FF4
:101CC0008327C10083A787041387F7FF8327C100F9
:101CD00023A4E7048327C10083A78704E348F0F81F
:101CE0006F008000130000008327C1001307F0FF7E
:101CF00023A4E704EF20904EEF20504A6F00000429
:101D00008327C10083A70701638207048327C100DB
:101D10009387070113850700EF10905F9307050075
:101D200063840700EF2080188327C10083A747043E
:101D30001387F7FF8327C10023A2E7048327C1008D
:101D400083A74704E34EF0FA6F0080001300000001
:101D50008327C1001307F0FF23A2E704EF201048F8
:101D6000130000008320C1011301010267800000FD
:101D7000130101FD232611022326A100EF201042AA
:101D80008327C10083A78703639807009307100088
:101D9000232EF1006F008000232E0100EF2010445D
:101DA0008327C101138507008320C10213010103AA
:101DB00067800000130101FE2326A1008327C100D4
:101DC00063960700737004306F0000008327C10022
:101DD00083A787036398070093071000232EF10061
:101DE0006F008000232E01008327C10113850700A7
:101DF0001301010267800000130101FD2326110277
:101E00002326A100EF2090398327C10003A7870371
:101E10008327C10083A7C7036318F7009307100047
:101E2000232EF1006F008000232E0100EF20103BD5
:101E30008327C101138507008320C1021301010319
:101E400067800000130101FE2326A1008327C10043
:101E500063960700737004306F0000008327C10091
:101E600003A787038327C10083A7C7036318F7006D
:101E700093071000232EF1006F008000232E010035
:101E80008327C10113850700130101026780000049
:101E9000130101FE2326A1002324B100232E0100FB
:101EA0006F008006178703001307C7868327C101C9
:101EB00093973700B307F70083A7070063900704E1
:101EC00017870300130707858327C10193973700FE
:101ED000B307F7000327810023A0E700178703005B
:101EE000130747838327C10193973700B307F70090
:101EF0000327C10023A2E7006F00C0018327C101AF
:101F000093871700232EF1000327C1019307700068
:101F1000E3FAE7F8130000001301010267800000F4
:101F2000130101FE2326A100232E01006F00C0042F
:101F3000177703001307077E8327C10193973700A4
:101F4000B307F70083A747000327C1006310F70218
:101F5000177703001307077C8327C1019397370086
:101F6000B307F70023A007006F00C0018327C1015A
:101F700093871700232EF1000327C10193077000F8
:101F8000E3F8E7FA13000000130101026780000084
:101F9000130101FD232611022326A1002324B100F1
:101FA0002322C1008327C100232EF100EF20101F40
:101FB0008327C10103A747049307F0FF6316F700C7
:101FC0008327C10123A207048327C10103A7870434
:101FD0009307F0FF6316F7008327C10123A40704CA
:101FE000EF20D01F8327C10183A78703639E0700CB
:101FF0008327C1019387470203264100832581007F
:1020000013850700EF1050250325C101EFF0DFC451
:10201000130000008320C102130101036780000048
:10202000130101FD232611022326A100130600003F
:10203000930540000325C100EFE05FB2232EA1000D
:102040008327C101138507008320C1021301010307
:1020500067800000130101FD232611022326A10041
:102060002324B100EF2090138327C10083A74705E5
:1020700063860700232E01006F00C0028327C10082
:1020800083A7870363860700232E01006F0080016A
:102090008327C1000327810023AAE70493071000C8
:1020A000232EF100EF2090138327C1011385070031
:1020B0008320C1021301010367800000130101FDA9
:1020C000232611022326A1002324B1008327C10067
:1020D000232CF1008327810183A747050327810073
:1020E0006306F700232E01006F00000383278101A0
:1020F00083A7870363860700232E01006F00C001BA
:10210000EF20D0098327810123AA0704EF20100DB7
:1021100093071000232EF1008327C10113850700C8
:102120008320C1021301010367800000130101FD38
:10213000232611022326A1002324B100232E01000F
:102140009307C101930600000326810093850700D1
:102150000325C100EFF00FB18327C10113850700EC
:102160008320C1021301010367800000130101FDF8
:10217000232611022326A100232E01009307C1016B
:1021800013060000938507000325C100EFF08FD5EB
:102190008327C101138507008320C10213010103B6
:1021A00067800000130101FD232611022326A100F0
:1021B0002324B1008327C10083A74705232CF10006
:1021C000232E01008327810163960700737004307A
:1021D0006F0000008327810103A787038327810104
:1021E00083A7C7036366F700737004306F000000B5
:1021F0008327810103A787038327810183A7C7035F
:102200006378F7069307C1000326810093850700D2
:1022100003258101EFF05F83232EA1008327810135
:1022200003A787049307F0FF631AF702832781014E
:1022300083A74702638E07028327810193874702A2
:1022400013850700EF10D00C930705006382070287
:1022500093071000232EF1006F0080018327810176
:1022600083A78704138717008327810123A4E7042A
:102270008327C101138507008320C10213010103D5
:1022800067800000130101FC232E1102232EA10000
:10229000232CB1002328D1002326E1002324F100C0
:1022A000232201012320110193070600231BF100C3
:1022B0008327C10163960700737004306F0000002C
:1022C0000327C1009307900063F6E70073700430A2
:1022D0006F000000835761018325410013850700CB
:1022E000EF10D07E2324A102832781026386071C7E
:1022F0008327810203A7070383566101B7070040C4
:102300009387F7FFB387F60093972700B307F7008B
:102310002322F1028327410293F7C7FF2322F10210
:102320008327410293F737006386070073700430F8
:102330006F000000835761011387070083260100A7
:102340000326C1008325810103258102EF1050413E
:10235000032601018325C10103254102EFE08FBC63
:10236000130705008327810223A0E700832781004C
:1023700063880700832781000327810223A0E700E9
:10238000EF20C06197E701009387072383A7070029
:102390001387170097E701009387072223A0E70020
:1023A00097E701009387470383A707006398070215
:1023B00097E70100938747020327810223A0E700E4
:1023C00097E701009387471F03A7070093071000B3
:1023D0006312F704EF10904B6F00C00397E7010002
:1023E0009387471E83A707006396070297E70100BC
:1023F000938787FE83A7070083A7C7020327C1002F
:10240000636AF70097E70100938707FD03278102BE
:1024100023A0E70097E701009387C71B83A7070066
:102420001387170097E701009387C71A23A0E700D7
:1024300097E701009387071A03A707008327810204
:1024400023A4E7048327810203A7C70297E70100BB
:102450009387071783A7070063FCE70083278102A0
:1024600003A7C70297E701009387871523A0E7001A
:102470008327810203A7C7029307070093972700CA
:10248000B387E7009397270017E70100130747FF7B
:102490003387E700832781029387470093850700EE
:1024A00013050700EFE08FBA930710002326F1020F
:1024B000EF20C0526F00C0009307F0FF2326F10207
:1024C0000327C102930710006318F70297E7010082
:1024D0009387470F83A707006380070297E70100F0
:1024E000938787EF83A7070083A7C7020327C1004D
:1024F00063F4E700EFE0CF898327C102138507006B
:102500008320C1031301010467800000130101FD52
:10251000232611022326A100EF2040488327C10073
:10252000639A070097E70100938707EB83A70700EB
:102530006F0080008327C100232EF1008327C10193
:102540009387470013850700EFE08FC48327C101FD
:1025500083A78702638A07008327C10193878701C6
:1025600013850700EFE0CFC28327C101938747009F
:102570009385070017E5010013054501EFE00FAD56
:1025800097E701009387C70183A707001387170008
:1025900097E701009387C70023A0E70097E70100B2
:1025A0009387470383A707001387170097E7010066
:1025B0009387470223A0E700EF20404297E70100FE
:1025C0009387470083A707006382070497E701000A
:1025D000938787E083A707000327C1016312F702EF
:1025E00097E70100938787FF83A7070063860700AB
:1025F000737004306F000000EFD09FF96F0000018E
:10260000EF20C039EF208001EF20403D1300000093
:102610008320C1021301010367800000130101FD43
:10262000232611022326A1002324B100232E01001A
:102630008327C10063960700737004306F000000A9
:102640008327810063960700737004306F000000D9
:1026500097E70100938787F883A707006386070041
:10266000737004306F000000EF00101D97E7010049
:102670009387C7F483A70700232CF1008327C100A9
:1026800083A7070003278100B307F700232AF1007F
:102690008327C10083A70700032781016376F70220
:1026A0008327C10083A70700032741016370F70454
:1026B000032741018327810163FAE7029307100092
:1026C000232EF1006F0080028327C10083A707003B
:1026D000032741016368F700032741018327810134
:1026E00063F6E70093071000232EF1008327C10053
:1026F0000327410123A0E7008327C101638207026A
:1027000097E70100938747CD83A70700938747008A
:1027100013850700EFE0CFA703254101EF10502FED
:10272000EF00D0132328A100832701016394070041
:10273000EFD01FE6130000008320C1021301010344
:1027400067800000130101FD232611022326A1004A
:10275000232E01008327C1006380070697E701004D
:102760009387C7E783A70700638607007370043069
:102770006F000000EF00500C97E70100938707E41B
:1027800083A707000327C100B307F700232CF1003C
:1027900097E70100938747C483A707009387470003
:1027A00013850700EFE0CF9E03258101EF1050262F
:1027B000EF00D00A232EA1008327C10163940700F4
:1027C000EFD01FDD130000008320C10213010103BD
:1027D00067800000130101FD232611022326A100BA
:1027E0008327C100232CF100832781016396070012
:1027F000737004306F00000097E701009387C7BD36
:1028000083A70700032781016316F700232E010029
:102810006F00400AEF2080188327810183A74701BA
:10282000232AF100EF20801B97E70100938747D40C
:1028300083A7070003274101630CF70097E7010016
:10284000938747D383A70700032741016318F70045
:1028500093072000232EF1006F00C00503274101DC
:1028600097E70100938707D46314F7028327810158
:1028700083A787026398070093073000232EF10097
:102880006F00400393072000232EF1006F008002A9
:102890000327410197E70100938747CF6318F700AB
:1028A00093074000232EF1006F00C0009307100033
:1028B000232EF1008327C101138507008320C10265
:1028C0001301010367800000130101FD232611029B
:1028D0002326A100EF20800C8327C100639A070004
:1028E00097E70100938747AF83A707006F00800039
:1028F0008327C100232EF1008327C10183A7C702CC
:10290000232CF100EF20800D832781011385070020
:102910008320C1021301010367800000130101FD40
:10292000232611022326A100EFD0DFDD9307050047
:10293000232EF1008327C100639A070097E7010067
:10294000938787A983A707006F0080008327C100B2
:10295000232CF1008327810183A7C702232AF100DA
:102960008327C10113850700EFD01FD883274101BA
:10297000138507008320C102130101036780000053
:10298000130101FD232611022326A1002324B100F7
:10299000232E0100032781009307900063F6E700D0
:1029A000737004306F0000000327810093079000CC
:1029B00063F6E700930790002324F100EF10107EE8
:1029C0008327C100639A070097E701009387C7A098
:1029D00083A707006F0080008327C100232CF1002C
:1029E0008327810183A70705232AF10003274101DB
:1029F00083278100630EF716032781008327410197
:102A000063FEE70297E701009387079D83A707000E
:102A1000032781016302F70497E701009387C79BAF
:102A200083A7070083A7C702032781006366F70215
:102A300093071000232EF1006F00000297E70100BA
:102A40009387879983A70700032781016316F700FF
:102A500093071000232EF1008327810183A7C7026B
:102A60002328F1008327810103A70705832781011C
:102A700083A7C7026318F70083278101032781001A
:102A800023A6E702832781010327810023A8E70407
:102A90008327810183A7870163CC07001307A00068
:102AA000832781003307F7408327810123ACE700A8
:102AB0008327810183A647010327010193070700AC
:102AC00093972700B387E7009397270017E7010044
:102AD0001307079BB387E7006396F6009307100080
:102AE0006F00800093070000638C07068327810135
:102AF0009387470013850700EFD09FE98327810163
:102B000003A7C70297E70100938787AB83A7070056
:102B100063FCE7008327810103A7C70297E7010051
:102B2000938707AA23A0E7008327810103A7C70291
:102B30009307070093972700B387E7009397270031
:102B400017E701001307C7933387E7008327810145
:102B5000938747009385070013050700EFD01FCF29
:102B60000327C101930710006314F700EFD05FA2A1
:102B7000EF10D066130000008320C102130101038F
:102B800067800000130101FD232611022326A10006
:102B9000EF10D0608327C100639A070097E7010018
:102BA0009387878383A707006F0080008327C10076
:102BB000232EF1008327C101938747001385070067
:102BC000EFD01FDD8327C10183A78702638A070037
:102BD0008327C1019387870113850700EFD05FDB4F
:102BE0008327C101938747009385070017E50100FC
:102BF0001305459BEFD09FC5EF10505E97D701009E
:102C00009387877D83A707000327C1016314F70615
:102C100097E701009387079B83A70700638207025A
:102C200097E701009387879B83A7070063860700C8
:102C3000737004306F000000EFD09F956F00400567
:102C400097E701009387079603A7070097E701001E
:102C50009387879683A70700631AF70097D7010029
:102C60009387877723A007006F008002EF009028EA
:102C70006F00000297E701009387C79483A70700BE
:102C800063880700EF109051EF105019EF101055A6
:102C9000130000008320C1021301010367800000BC
:102CA000130101FE2326A100232E01008327C1006A
:102CB000232CF1008327C100639607007370043052
:102CC0006F0000008327810103A7470197E70100F8
:102CD0009387478D6316F700930710006F008000FD
:102CE00093070000638E07028327810103A78702F1
:102CF00097E70100938747886304F70283278101E0
:102D000083A7870263960700930710006F00800077
:102D1000930700006386070093071000232EF1003D
:102D20008327C1011385070013010102678000009A
:102D3000130101FD232611022326A1008327C100D0
:102D4000232EF1008327C1006396070073700430BF
:102D50006F0000008327C1016384070C97D701002F
:102D60009387876783A707000327C101630AF70AD0
:102D7000EF10D0420325C101EFF09FF213070500C9
:102D800093071000631CF7088327C101938747004E
:102D900013850700EFD0DFBF8327C10103A7C70258
:102DA00097E701009387C78183A7070063FCE700CB
:102DB0008327C10103A7C70297E7010093874780D4
:102DC00023A0E7008327C10103A7C70293070700D9
:102DD00093972700B387E7009397270017D7010041
:102DE0001307076A3387E7008327C10193874700EA
:102DF0009385070013050700EFD05FA58327C10166
:102E000003A7C70297D701009387075D83A7070031
:102E100083A7C7026364F700EFD08FF7EF10103C71
:102E2000130000008320C10213010103678000002A
:102E3000130101FD232611022326A100232E0100E8
:102E40008327C100232CF1008327C100639607006C
:102E5000737004306F000000EFD0DF8A9307050025
:102E6000232AF10003258101EFF09FE313070500FA
:102E7000930710006314F70C97D701009387077628
:102E800083A707006390070A8327810103A7C7026E
:102E900097D701009387475483A7070083A7C702EA
:102EA0006366F70093071000232EF100832781014A
:102EB0009387470013850700EFD09FAD83278101DB
:102EC00003A7C70297D701009387876F83A70700DF
:102ED00063FCE7008327810103A7C70297D701009E
:102EE0009387076E23A0E7008327810103A7C7020A
:102EF0009307070093972700B387E700939727006E
:102F000017D701001307C7573387E70083278101CD
:102F1000938747009385070013050700EFD01F93A1
:102F20006F00C00183278101938787019385070084
:102F300017D5010013054564EFD05F918327410148
:102F400013850700EFD04FFA8327C10113850700CF
:102F50008320C1021301010367800000130101FEF9
:102F6000232E1100930800001308000093070000AF
:102F700013070000930600001306004097D50100D8
:102F80009385450817150000130505FBEFF08FAF7B
:102F90002326A1000327C100930710006316F70042
:102FA000EF20C03A2326A1000327C1009307100099
:102FB000631EF7027370043097D701009387C761CF
:102FC0001307F0FF23A0E70097D701009387875FDF
:102FD0001307100023A0E70097D701009387075E2F
:102FE00023A00700EFD00FC06F0040018327C1006E
:102FF00063960700737004306F0000001300000038
:103000008320C1011301010267800000130101FF49
:10301000232611007370043097D701009387875AD5
:1030200023A00700EFD04FCE130000008320C10083
:10303000130101016780000097D701009387075AA9
:1030400083A707001387170097D7010093870759B5
:1030500023A0E7001300000067800000130101FEB9
:10306000232E11002326010097D7010093870757CD
:1030700083A7070063960700737004306F00000099
:10308000EF10D01197D701009387475583A707000A
:103090001387F7FF97D701009387475423A0E700D2
:1030A00097D701009387875383A707006394071678
:1030B00097D701009387475083A70700638C0714B5
:1030C0006F00800C97D701009387074B83A7C70039
:1030D00083A7C7002324F1008327810093878701FA
:1030E00013850700EFD0DF8A83278100938747008D
:1030F00013850700EFD0DF898327810003A7C7026C
:1031000097D701009387C74B83A7070063FCE700AD
:103110008327810003A7C70297D701009387474AF7
:1031200023A0E7008327810003A7C70293070700B6
:1031300093972700B387E7009397270017D70100DD
:10314000130707343387E7008327810093874700FD
:103150009385070013050700EFD04FEF8327810009
:1031600003A7C70297D701009387072783A7070004
:1031700083A7C702636AF70097D7010093870745C3
:103180001307100023A0E70097D701009387C73EDD
:1031900083A70700E39807F297D701009387C742F8
:1031A00083A70700638807046F00C003EF00002BAC
:1031B00093070500638A070097D7010093870741AB
:1031C0001307100023A0E70097D701009387C73F9C
:1031D00083A707001387F7FF97D701009387C73EA0
:1031E00023A0E70097D701009387073E83A7070036
:1031F000E39E07FA97D701009387473D03A707008F
:10320000930710006318F700930710002326F100BE
:10321000EFD00FB8EF10807C8327C1001385070023
:103220008320C1011301010267800000130101FE28
:10323000232E1100EF10807697D70100938707386F
:1032400083A707002326F100EF1040798327C100F0
:10325000138507008320C10113010102678000006C
:10326000130101FE232E1100EFD0CFC993070500F3
:103270002326F10097D701009387473483A70700DF
:103280002324F1008327C10013850700EFD0CFC5A9
:1032900083278100138507008320C10113010102E8
:1032A0006780000097D701009387073183A7070045
:1032B0001385070067800000130101FD232611021A
:1032C0002326A1002324B1002322C100232E0100C4
:1032D0009307A000232CF100EFF01FD697D7010031
:1032E0009387872D83A7070003278100636CF7145A
:1032F000832781019387F7FF232CF1008327C101E6
:10330000939757000327C100B306F70003278101F5
:103310009307070093972700B387E7009397270049
:1033200017D701001307C715B387E700130610006E
:103330009385070013850600EF108004130705002E
:103340008327C101B387E700232EF1008327810182
:10335000E39007FA8327C101939757000327C10021
:103360003307F70097D701009387872083A70700CB
:10337000130620009385070013050700EF10400097
:10338000130705008327C101B387E700232EF1004F
:103390008327C101939757000327C1003307F70024
:1033A00097D701009387071D83A707001306200006
:1033B0009385070013050700EF00907C13070500B5
:1033C0008327C101B387E700232EF1008327C101C2
:1033D000939757000327C100B307F7001306400077
:1033E00097D501009385851A13850700EF00507962
:1033F000130705008327C101B387E700232EF100DF
:103400008327C101939757000327C100B307F70033
:103410001306300097D501009385C5181385070062
:10342000EF001076130705008327C101B387E7007B
:10343000232EF10083274100638607008327410084
:1034400023A00700EFF09FC18327C1011385070068
:103450008320C1021301010367800000130101FDF5
:1034600023261102232E010097D701009387071707
:1034700083A70700639C072297D70100938707144F
:1034800083A707001387170097D7010093870713B7
:1034900023A0E70097D701009387471283A707006F
:1034A000232CF10083278101639C070697D7010035
:1034B0009387070C83A7070083A70700638607008D
:1034C000737004306F00000097D701009387470A9C
:1034D00083A70700232AF10097D701009387870964
:1034E00003A7070097D701009387870823A0E70069
:1034F00097D70100938707080327410123A0E7001E
:1035000097D701009387C70C83A70700138717007D
:1035100097D701009387C70B23A0E700EF10001097
:1035200097D701009387470B83A7070003278101E3
:10353000636CF71297D701009387870383A707006F
:1035400083A7070063960700930710006F008000B1
:1035500093070000638C070097D701009387C70784
:103560001307F0FF23A0E7006F00001097D70100BA
:103570009387070083A7070083A7C70083A7C70017
:103580002328F1008327010183A747002326F100A8
:10359000032781018327C100637CF70097D70100CF
:1035A000938787030327C10023A0E7006F00C00BA8
:1035B000832701019387470013850700EFD04FBD94
:1035C0008327010183A78702638A070083270101FC
:1035D0009387870113850700EFD08FBB83270101F5
:1035E00003A7C70297D70100938787FD83A707002A
:1035F00063FCE7008327010103A7C70297D70100F7
:10360000938707FC23A0E7008327010103A7C702D4
:103610009307070093972700B387E7009397270046
:1036200017D701001307C7E53387E7008327010198
:10363000938747009385070013050700EFD00FA17C
:103640008327010103A7C70297D701009387C7D833
:1036500083A7070083A7C702E36EF7EC9307100068
:10366000232EF1006FF01FED97D701009387C7D687
:1036700083A7070003A7C70297D60100938646E0F9
:103680009307070093972700B387E70093972700D6
:10369000B387F60003A707009307100063F6E7025D
:1036A00093071000232EF1006F00000297D701004E
:1036B000938787F183A707001387170097D7010027
:1036C000938787F023A0E70097D70100938707F03F
:1036D00083A707006386070093071000232EF100DD
:1036E0008327C101138507008320C1021301010351
:1036F00067800000130101FE232E110097D70100FF
:103700009387C7ED83A70700638C070097D7010055
:103710009387C7EB1307100023A0E7006F00C018C2
:1037200097D70100938787EA23A0070097D7010066
:10373000938787CA83A7070083A707032326F1007F
:10374000B7A7A5A59387575A2324F1008327C10063
:1037500083A70700032781006310F7048327C100B4
:103760009387470083A70700032781006316F702AA
:103770008327C1009387870083A707000327810061
:10378000631CF7008327C1009387C70083A7070046
:10379000032781006302F70697D701009387C7C309
:1037A00003A7070097D70100938707C383A70700E4
:1037B000938747039385070013050700EF40002117
:1037C0006F00800397D70100938787DF83A70700E7
:1037D00063960700737004306F00000097D70100F4
:1037E000938707DE83A707001387F7FF97D70100AA
:1037F000938707DD23A0E70097D70100938747DC75
:1038000003A7070097D60100938686C79307070092
:1038100093972700B387E70093972700B387F600B5
:1038200083A70700E38007FA97D70100938747D95A
:1038300003A707009307070093972700B387E700C4
:103840009397270017D70100130787C3B387E700B3
:103850002322F1008327410083A7470003A74700E5
:103860008327410023A2E7008327410003A74700E5
:103870008327410093878700631CF700832741005B
:1038800083A7470003A747008327410023A2E7003F
:103890008327410083A7470003A7C70097D70100EC
:1038A000938787B323A0E700130000008320C101A2
:1038B0001301010267800000130101FD232611029C
:1038C0002326A1002324B1008327C10063960700AB
:1038D000737004306F00000097D701009387C7AF63
:1038E00083A7070093878701938507000325C100FD
:1038F000EFC09FFD97D70100938707AE83A707000E
:103900009387470013850700EFD08F880327810036
:103910009307F0FF6314F70297D701009387C7ABB3
:1039200083A70700938747009385070017D50100F9
:10393000130545C7EFC09FF16F00400297D7010004
:103940009387C7C783A7070003278100B307F70042
:10395000232EF1000325C101EF00900B130000009E
:103960008320C1021301010367800000130101FDE0
:10397000232611022326A1002324B1002322C10003
:103980008327C10063960700737004306F00000046
:1039900097D70100938787C483A707006396070022
:1039A000737004306F00000097D701009387C7A29F
:1039B00083A70700832681003707008033E7E600EE
:1039C00023ACE70097D70100938707A183A70700DF
:1039D00093878701938507000325C100EFC01FE788
:1039E00097D701009387479F83A7070093874700D6
:1039F00013850700EFC0DFF9032741009307F0FFAD
:103A00006314F70297D701009387079D83A70700E8
:103A1000938747009385070017D50100130585B8E4
:103A2000EFC0DFE26F00400297D70100938707B92C
:103A300083A7070003274100B307F700232EF100F7
:103A40000325C101EF00C07C130000008320C102E8
:103A50001301010367800000130101FD23261102F9
:103A60002326A1002324B1002322C1008327C10003
:103A700063960700737004306F00000097D7010051
:103A80009387879583A7070093878701938507000E
:103A90000325C100EFC09FDB97D701009387C79331
:103AA00083A707009387470013850700EFC05FEEE9
:103AB00003274100930710006314F70297D7010012
:103AC0009387879183A70700938747009385070013
:103AD00017D50100130505ADEFC05FD76F00400299
:103AE00097D70100938787AD83A70700032781003D
:103AF000B307F700232EF1000325C101EF00407149
:103B0000130000008320C10213010103678000003D
:103B1000130101FD232611022326A1008327C100E2
:103B200083A7C70083A7C700232CF1008327810147
:103B300063960700737004306F00000083278101D3
:103B40009387870113850700EFC09FE497D7010093
:103B50009387C7A883A70700639E07068327810171
:103B60009387470013850700EFC09FE283278101F9
:103B700003A7C70297D70100938787A483A70700ED
:103B800063FCE7008327810103A7C70297D70100E1
:103B9000938707A323A0E7008327810103A7C70218
:103BA0009307070093972700B387E70093972700B1
:103BB00017D701001307C78C3387E70083278101DC
:103BC000938747009385070013050700EFC01FC8C0
:103BD0006F00C001832781019387870193850700C8
:103BE00017D5010013054599EFC05FC683278101F2
:103BF00003A7C70297C701009387077E83A7070023
:103C000083A7C70263F0E70293071000232EF10099
:103C100097D701009387879B1307100023A0E70025
:103C20006F008000232E01008327C1011385070048
:103C30008320C1021301010367800000130101FD0D
:103C4000232611022326A1002324B10097D70100C7
:103C50009387C79883A707006396070073700430A3
:103C60006F00000003278100B70700803367F7006B
:103C70008327C10023A0E7008327C10083A7C700D3
:103C8000232CF100832781016396070073700430B1
:103C90006F0000000325C100EFC09FCF8327810183
:103CA0009387470013850700EFC09FCE83278101CC
:103CB00003A7C70297D701009387879083A70700C0
:103CC00063FCE7008327810103A7C70297D70100A0
:103CD0009387078F23A0E7008327810103A7C702EB
:103CE0009307070093972700B387E7009397270070
:103CF00017C701001307C7783387E70083278101BF
:103D0000938747009385070013050700EFC01FB492
:103D10008327810103A7C70297C701009387C76B59
:103D200083A7070083A7C70263F0E7029307100089
:103D3000232EF10097D701009387478913071000BE
:103D400023A0E7006F008000232E01008327C1011C
:103D5000138507008320C10213010103678000005F
:103D6000130101FF2326A1008327C10063960700EA
:103D7000737004306F00000097D701009387478568
:103D800003A707008327C10023A0E70097D70100FE
:103D90009387C78203A707008327C10023A2E700F8
:103DA000130000001301010167800000130101FDF1
:103DB000232611022326A1002324B1008327C1005A
:103DC00063960700737004306F0000008327810042
:103DD00063960700737004306F000000EF00103C22
:103DE00097C701009387877D83A70700232CF100E5
:103DF0008327810003A707009307F0FF6316F700EE
:103E0000232E01006F0000098327C10003A70700CC
:103E100097C701009387C77B83A707006300F7025A
:103E20008327C10083A74700032781016368F70048
:103E300093071000232EF1006F00C0058327C100F7
:103E400083A74700032781013307F74083278100B9
:103E500083A70700637CF7028327810003A707007D
:103E60008327C10083A6470083278101B387F640DB
:103E70003307F7008327810023A0E7000325C10053
:103E8000EFF01FEE232E01006F00C000930710001B
:103E9000232EF100EF0090348327C1011385070022
:103EA0008320C102130101036780000097C701004E
:103EB0009387C7711307100023A0E70013000000C9
:103EC00067800000130101FE2326A1008327C100A3
:103ED000638E07008327C100232CF1008327810113
:103EE00083A7C704232EF1006F008000232E01005A
:103EF0008327C101138507001301010267800000B9
:103F0000130101FE2326A1002324B1008327C10051
:103F1000638C07008327C100232EF1008327C10192
:103F20000327810023A6E704130000001301010208
:103F300067800000130101FE232E11002326A1003B
:103F4000EF00002197C701009387875303A707005D
:103F500093071000E3F6E7FEEFC08FE36FF05FFE1C
:103F6000130101FC232E1102232EA100232CB100EA
:103F7000232AC1002328D100930707002317F1004B
:103F8000232601026F004004032781018327C10219
:103F9000B307F70003C707008326C1018327C102C7
:103FA000B387F600238AE702032781018327C10232
:103FB000B307F70083C70700638007028327C102A6
:103FC000938717002326F1020327C1029307F0000D
:103FD000E3FCE7FA6F008000130000008327C101B3
:103FE000A3810704032741019307900063F6E700CC
:103FF00093079000232AF1008327C1010327410181
:1040000023A6E7028327C1010327410123A8E70470
:104010008327C10123AA07048327C101938747008F
:1040200013850700EFC0DF808327C10193878701D5
:1040300013850700EFC0CFFF8327C1010327C1010C
:1040400023A8E7001307A000832741013307F740A7
:104050008327C10123ACE7008327C1010327C101E6
:1040600023A2E7028327C10123A207048327C101FA
:1040700023AC07048327C10123AE0704130000000B
:104080008320C1031301010467800000130101FEB6
:10409000232E1100232601006F0080030327C10097
:1040A0009307070093972700B387E70093972700AC
:1040B00017C701001307C73CB387E7001385070044
:1040C000EFC08FF18327C100938717002326F100EB
:1040D0000327C10093079000E3F2E7FC17C5010036
:1040E00013058546EFC04FEF17C5010013050547BF
:1040F000EFC08FEE17C5010013050548EFC0CFEDE7
:1041000017C5010013058548EFC00FED17C5010065
:1041100013054549EFC04FEC97C70100938747450A
:1041200017C701001307474223A0E70097C7010004
:104130009387474417C701001307474223A0E700AE
:10414000130000008320C1011301010267800000F9
:10415000130101FE232E11006F008009EFE0DFED57
:1041600097C701009387874283A7070093B717007B
:1041700093F7F70F2326F100EFE05FEE8327C100EE
:1041800063980706EF00900197C7010093870740E7
:1041900083A7C70083A7C7002324F10083278100DA
:1041A0009387470013850700EFC08FFE97C7010074
:1041B0009387874083A707001387F7FF97C70100FE
:1041C0009387873F23A0E70097C701009387473D68
:1041D00083A707001387F7FF97C701009387473C22
:1041E00023A0E700EF00807F03258100EF00C03FA0
:1041F00097C701009387C73A83A70700E39007F6A4
:10420000130000008320C101130101026780000038
:10421000130101FE232E11002326A10097C70100E0
:104220009387871B83A707000327C10023A2E7000A
:1042300097C701009387873883A707000327C1002A
:104240006378F70297C701009387C73203A7070077
:1042500097C701009387471883A7070093874700F4
:104260009385070013050700EFC00FE66F000005F8
:1042700097C701009387C72F03A7070097C70100BF
:104280009387871583A707009387470093850700C7
:1042900013050700EFC04FE397C701009387C733AB
:1042A00083A707000327C100637AF70097C70100BF
:1042B000938787320327C10023A0E7001300000083
:1042C0008320C1011301010267800000130101FD79
:1042D00023261102930705002324B1002317F100C0
:1042E00083278100639E07008357E100939727008F
:1042F00013850700EF20C02E930705006F00800094
:1043000083278100232CF10083278101638A070220
:1043100013050006EF20C02C232EA1008327C10126
:10432000638A07008327C1010327810123A8E702CD
:104330006F00400103258101EF20404A6F0080009B
:10434000232E01008327C101638207028327C10155
:1043500003A707038357E1009397270013860700FD
:104360009305500A13050700EF20006A8327C10157
:10437000138507008320C102130101036780000039
:10438000130101FC232E1102232C81022326A100FC
:104390002324B1002322C1002326010283278100A8
:1043A00083A707006388071C832781002324F10269
:1043B0008327810283A7470003A747008327810241
:1043C00023A2E7008327810203A7470083278102F6
:1043D00093878700631CF7008327810283A7470028
:1043E00003A747008327810223A2E70083278102D6
:1043F00083A7470083A7C7002322F10283278100F8
:104400002320F1028327010283A7470003A7470067
:104410008327010223A2E7008327010203A74700A5
:104420008327010293878700631CF700832701021B
:1044300083A7470003A747008327010223A2E700C1
:104440008327010283A7470083A7C700232EF1001B
:104450008327C102939757000327C100B307F700D2
:104460000327C10123A0E7008327C10293975700C8
:104470000327C100B307F7000327C1011307470350
:1044800023A2E7008327C102939757000327C100A7
:10449000B307F7000327C1010327870423A4E7001C
:1044A0008327C102939757000327C100B307F70082
:1044B0000327410023A6E7008327C10293975700F3
:1044C0000327C100B307F7000327C1010327C70271
:1044D00023A8E70003274100930730006314F70285
:1044E0008327C10183A78702638E07008327C10248
:1044F000939757000327C100B307F7001307200065
:1045000023A6E7008327C102939757000327C10022
:10451000B307F7000327C1010327070523AAE70014
:104520008327C102939757000327C100B307F70001
:1045300023AC07008327C10183A607038327C10299
:10454000939757000327C1003304F7001385060033
:10455000EF00C00393070500231EF4008327C10268
:10456000938717002326F1020327C1018327410205
:10457000E316F7E88327C102138507008320C103F0
:10458000032481031301010467800000130101FE6D
:104590002326A100232E01006F00C0018327C10044
:1045A000938717002326F1008327C1019387170003
:1045B000232EF1008327C10003C707009307500A89
:1045C000E30EF7FC8327C10193D72700232EF100C8
:1045D0008327C1019397070193D70701138507002C
:1045E0001301010267800000130101FE232E110058
:1045F0002326A1008327C10083A707031385070093
:10460000EF20C01D0325C100EF20401D1300000056
:104610008320C1011301010267800000130101FF23
:1046200097C701009387C7F483A7070083A70700F4
:1046300063960700930710006F0080009307000047
:10464000638C070097C70100938707F91307F0FFF2
:1046500023A0E7006F00000397C70100938747F18D
:1046600083A7070083A7C70083A7C7002326F100FD
:104670008327C10003A7470097C701009387C7F5A9
:1046800023A0E70013000000130101016780000070
:10469000130101FF97C70100938707D483A7070081
:1046A0002326F1008327C1001385070013010101B0
:1046B00067800000130101FF97C70100938787F00F
:1046C00083A7070063980700930710002326F100D3
:1046D0006F00400297C70100938747F083A7070048
:1046E00063980700930720002326F1006F008000E5
:1046F000232601008327C100138507001301010150
:1047000067800000130101FD232611022326A1006A
:104710008327C100232EF1008327C100638A07127B
:104720008327C10103A7C70297C701009387C7CAA0
:1047300083A7070083A7C702637CF7108327C10103
:1047400083A7870163C2070297C701009387C7C881
:1047500083A7070083A7C7021307A0003307F7400A
:104760008327C10123ACE7008327C10183A647014A
:104770008327C10103A7C702930707009397270068
:10478000B387E7009397270017C70100130747CFA8
:10479000B387E7006396F600930710006F00800070
:1047A00093070000638A07088327C10193874700A6
:1047B00013850700EFC0CF9D97C701009387C7C13E
:1047C00083A7070003A7C7028327C10123A6E70227
:1047D0008327C10103A7C70297C70100938747DE5C
:1047E00083A7070063FCE7008327C10103A7C70273
:1047F00097C701009387C7DC23A0E7008327C10187
:1048000003A7C7029307070093972700B387E70022
:104810009397270017C70100130787C63387E70060
:104820008327C1019387470093850700130507007D
:10483000EFC0CF816F00C00197C701009387C7B950
:1048400083A7070003A7C7028327C10123A6E702A6
:10485000130000008320C1021301010367800000E0
:10486000130101FD232611022326A1008327C10085
:10487000232CF100232E01008327C100638607103B
:1048800097C70100938747B583A7070003278101D6
:104890006306F700737004306F0000008327810106
:1048A00083A7470563960700737004306F0000000C
:1048B0008327810183A747051387F7FF832781019A
:1048C00023AAE7048327810103A7C7028327810165
:1048D00083A70705630AF70A8327810183A7470592
:1048E0006394070A83278101938747001385070094
:1048F000EFC00F8A8327810103A707058327810162
:1049000023A6E7028327810183A7C7021307A0001C
:104910003307F7408327810123ACE7008327810118
:1049200003A7C70297C70100938787C983A707001A
:1049300063FCE7008327810103A7C70297C7010033
:10494000938707C823A0E7008327810103A7C70235
:104950009307070093972700B387E70093972700F3
:1049600017C701001307C7B13387E7008327810109
:10497000938747009385070013050700EFB01FEDED
:1049800093071000232EF1008327C1011385070030
:104990008320C1021301010367800000737004309B
:1049A00097C70100938707C283A7070063840702A4
:1049B00097C70100938747A283A7070003A747046F
:1049C0001307170023A2E70497C701009387C7A026
:1049D00083A70700130000006780000097C701004D
:1049E000938747BE83A707006384070497C7010026
:1049F0009387879E83A7070083A74704638A0702DC
:104A000097C701009387479D83A7070003A7470423
:104A10001307F7FF23A2E70497C701009387C79BFB
:104A200083A7070083A747046394070073600430DB
:104A30001300000067800000130101FF97C7010009
:104A40009387879983A7070083A787012326F1000F
:104A500097C701009387479883A7070003A7C7025A
:104A600097C701009387479783A707009306A00085
:104A70003387E64023ACE7008327C1001385070096
:104A8000130101016780000097C701009387C79455
:104A900083A70700638E070097C701009387C7931A
:104AA00083A7070003A747051307170023AAE704F6
:104AB00097C701009387479283A7070013850700D4
:104AC00067800000130101FD232611022326A100A7
:104AD0002324B100EFF09FEC97C701009387C78FA5
:104AE00083A7070083A787056396070897C7010078
:104AF0009387878E83A707001307100023AEE70470
:104B0000832781006388070697C701009387C78CB6
:104B100083A707009387470013850700EFB05FE77F
:104B2000032781009307F0FF6314F70297C7010082
:104B30009387878A83A70700938747009385070099
:104B400017C50100130505A6EFB05FD06F00400246
:104B500097C70100938787A683A7070003278100D3
:104B6000B307F700232EF1000325C101EFF04FEA50
:104B7000EFB01FA2EFF09FE6EFF05FE297C70100F2
:104B80009387878583A7070083A78705232CF100D8
:104B900083278101638C07028327C100638C070090
:104BA00097C701009387478383A7070023AC0704B7
:104BB0006F00C00197C701009387078283A7070092
:104BC00003A787051307F7FF23ACE70497C7010086
:104BD0009387878083A7070023AE0704EFF01FE0C9
:104BE00083278101138507008320C102130101037C
:104BF00067800000130101FD232611022326A10076
:104C00002324B1002322C1002320D100EFF01FD9BB
:104C100097B701009387477C83A7070003A7C705C1
:104C2000930720006306F70A97B701009387C77AB6
:104C300083A7070083A687050327C1001347F7FF53
:104C400033F7E60023ACE70497B701009387C778F2
:104C500083A707001307100023AEE7048327010092
:104C60006388070697B701009387077783A7070034
:104C70009387470013850700EFB09FD103270100FA
:104C80009307F0FF6314F70297B701009387C77487
:104C900083A70700938747009385070017C5010086
:104CA00013054590EFB09FBA6F00400297C701000F
:104CB0009387C79083A7070003270100B307F70076
:104CC000232CF10003258101EFF08FD4EFB05F8C2E
:104CD000EFF0DFD0EFF09FCC83274100638E070019
:104CE00097B701009387476F83A7070003A787053E
:104CF0008327410023A0E70097B701009387C76D82
:104D000083A7070003A7C705930710006316F700E2
:104D1000232E01006F00C00297B701009387C76B75
:104D200083A7070083A68705032781001347F7FFA2
:104D300033F7E60023ACE70493071000232EF100BD
:104D400097B701009387476983A7070023AE07043D
:104D5000EFF0DFC88327C101138507008320C1025C
:104D60001301010367800000130101FD23261102D6
:104D70002326A1002324B1002322C1002320D10037
:104D800093071000232EF1008327C10063960700CC
:104D9000737004306F0000008327C100232CF100E2
:104DA000EFF0DFBF83270100638A070083278101BB
:104DB00003A787058327010023A0E700832781013C
:104DC00083A7C705232AF100832781011307200049
:104DD00023AEE704032741009307400063ECE70894
:104DE000832741001397270097B701009387072275
:104DF000B307F70003A7070097B7010093870721C0
:104E0000B307F700678007008327810103A78705A1
:104E1000832781003367F7008327810123ACE704F0
:104E20006F0040058327810183A78705138717003B
:104E30008327810123ACE7046F00C003832781012E
:104E40000327810023ACE7046F00C0020327410160
:104E500093072000630AF70083278101032781005D
:104E600023ACE7046F000001232E01006F008000D7
:104E70001300000003274101930710006316F70A8F
:104E8000832781019387470013850700EFB05FB048
:104E90008327810103A7C70297B701009387477251
:104EA00083A7070063FCE7008327810103A7C702EC
:104EB00097B701009387C77023A0E700832781017C
:104EC00003A7C7029307070093972700B387E7005C
:104ED0009397270017B701001307875A3387E70016
:104EE00083278101938747009385070013050700F7
:104EF000EFB0DF958327810183A7870263860700D0
:104F0000737004306F0000008327810103A7C7027C
:104F100097B701009387474C83A7070083A7C70271
:104F200063F4E700EFB0CFE6EFF05FAB8327C1019A
:104F3000138507008320C10213010103678000006D
:104F4000130101FC232E1102232EA100232CB100FA
:104F5000232AC1002328D1002326E1009307100053
:104F60002326F1028327C101639607007370043082
:104F70006F0000008327C1012324F102EFB08FF8F6
:104F8000930705002322F10283270101638A0700AA
:104F90008327810203A787058327010123A0E70058
:104FA0008327810283A7C7052320F102832781027B
:104FB0001307200023AEE7040327410193074000B5
:104FC00063ECE708832741011397270097B7010097
:104FD00093870705B307F70003A7070097B70100FA
:104FE00093870704B307F7006780070083278102D0
:104FF00003A78705832781013367F7008327810291
:1050000023ACE7046F0040058327810283A787054F
:10501000138717008327810223ACE7046F00C003C6
:10502000832781020327810123ACE7046F00C002BC
:105030000327010293072000630AF70083278102F8
:105040000327810123ACE7046F000001232601023E
:105050006F00800013000000032701029307100077
:105060006314F70E8327810283A7870263860700F4
:10507000737004306F00000097B7010093870756E4
:1050800083A70700639E0706832781029387470053
:1050900013850700EFB0DF8F8327810203A7C702C4
:1050A00097B701009387C75183A7070063FCE70008
:1050B0008327810203A7C70297B701009387475050
:1050C00023A0E7008327810203A7C70293070700F5
:1050D00093972700B387E7009397270017B701003E
:1050E0001307073A3387E700832781029387470036
:1050F0009385070013050700EFB04FF56F00C0015F
:1051000083278102938787019385070017B50100E4
:1051100013058546EFB08FF38327810203A7C702EB
:1051200097B701009387472B83A7070083A7C70280
:1051300063FCE7008327C100638807008327C10061
:105140001307100023A0E7008327410213850700FF
:10515000EFB08FD98327C102138507008320C103D5
:105160001301010467800000130101FD23261102D1
:105170002326A1002324B1008327C10063960700E2
:10518000737004306F0000008327C100232EF100EC
:10519000EFB04FD793070500232CF1008327C101FF
:1051A00083A7C705232AF1008327C1011307200025
:1051B00023AEE7048327C10183A787051387170060
:1051C0008327C10123ACE7040327410193071000A3
:1051D0006314F70E8327C10183A787026386070044
:1051E000737004306F00000097B701009387073F8A
:1051F00083A70700639E07068327C10193874700A3
:1052000013850700EFB0CFF88327C10103A7C702BA
:1052100097B701009387C73A83A7070063FCE700AD
:105220008327C10103A7C70297B7010093874739B6
:1052300023A0E7008327C10103A7C7029307070044
:1052400093972700B387E7009397270017B70100CC
:10525000130707233387E7008327C101938747009C
:105260009385070013050700EFB04FDE6F00C00104
:105270008327C101938787019385070017B5010034
:105280001305852FEFB08FDC8327C10103A7C70269
:1052900097B701009387471483A7070083A7C70226
:1052A00063FCE70083278100638807008327810070
:1052B0001307100023A0E70083278101138507004F
:1052C000EFB08FC2130000008320C102130101035D
:1052D00067800000130101FD232611022326A1008F
:1052E0008327C100232CF10083278101639A0700E3
:1052F00097B701009387470E83A707006F008000D0
:1053000083278101232CF100EFF04FE983278101EE
:1053100003A7C70593072000631CF70083278101BB
:1053200023AE070493071000232EF1006F008000C6
:10533000232E0100EFF08FEA8327C10113850700B8
:105340008320C1021301010367800000130101FEE5
:10535000232E110023260100EF00500B97B7010008
:105360009387072B83A70700638A0702930800002F
:1053700013080000930700001307200093060000A5
:105380001306004097B501009385C5CA17050000B4
:105390001305852EEFC01FEF2326A1008327C10030
:1053A00063960700737004306F0000008327C1000C
:1053B000138507008320C1011301010267800000EB
:1053C000130101FC232E1102232EA100232CB10076
:1053D000232AC1002328D1002326E100832781014D
:1053E00063960700232601026F0080061305C002A2
:1053F000EF10001F2326A1028327C102638A07043E
:10540000EF00D0008327C1020327C10123A0E700DA
:105410008327C1020327810123ACE7008327C10250
:105420000327410123AEE7008327C10203270101BF
:1054300023A0E7028327C1020327C10023A2E702BA
:105440008327C1029387470013850700EFB04FBE43
:105450008327810163960700737004306F0000009A
:105460008327C102138507008320C10313010104B0
:1054700067800000130101FC232E1102232EA100DE
:10548000232CB100232AC1002328D1002326E100C8
:10549000232601028327C10163960700737004303D
:1054A0006F00000097B701009387871683A7070056
:1054B000638C070A832781012320F102832741019E
:1054C0002322F1028327C1012324F1020327810152
:1054D0009307500063C6E706EFF0CF9D1307050062
:1054E000930720006318F70297B7010093874712CC
:1054F00083A7070013070102930600000326C100DB
:105500009305070013850700EFB0DF9E2326A10255
:105510006F00800597B701009387870F83A7070067
:10552000130701029306000013060000930507000D
:1055300013850700EFB01F9C2326A1026F00C00255
:1055400097B701009387C70C83A7070013070102D1
:105550009306000003260101930507001385070049
:10556000EFB01FC02326A1028327C10213850700C5
:105570008320C1031301010467800000130101FEB1
:105580002326A1008327C100232EF1008327C10019
:1055900063960700737004306F0000008327C10119
:1055A00083A707001385070013010102678000002D
:1055B000130101FD232611022326A1002324B1009B
:1055C00097B701009387470483A7070083A7C70005
:1055D00083A7C700232EF1008327C10193874700CB
:1055E00013850700EFB0CFBA8327C10103A7C70116
:1055F000930710006310F7068327C10103A78701F3
:105600008327C100B307F7008326C100032681006A
:10561000938507000325C101EF00802213070500D1
:10562000930710006318F7021307000093060000A9
:105630000326C100930500000325C101EFF09FE39D
:10564000232CA10083278101639607007370043027
:105650006F0000008327C10183A747020325C10112
:10566000E7800700130000008320C102130101033B
:1056700067800000130101FD232611022326A100EB
:105680009307810113850700EF00800E232EA100F0
:1056900083278101938507000325C101EF00C00026
:1056A000EF0000286FF0DFFD130101FD232611023A
:1056B0002326A1002324B100EFD01F989307810176
:1056C00013850700EF004011232EA10083278101DD
:1056D0006396070883278100639207020327C100AE
:1056E0008327C10163ECE700EFD05F978325C101F9
:1056F0000325C100EFF0DFEB6F00800683278100F8
:105700006380070297B70100938747F083A70700DC
:1057100083A7070093B7170093F7F70F2324F1002F
:1057200097B701009387C7EE83A607000327C10040
:105730008327C101B307F740032681009385070043
:1057400013850600EFC0DF84EFD05F91930705005B
:1057500063980700EFA0DFE36F008000EFD01F9099
:10576000130000008320C1021301010367800000C1
:10577000130101FE2326A10097B701009387C7E814
:1057800083A7070083A7070093B7170093F7F70FC6
:10579000138707008327C10023A0E7008327C100E8
:1057A00083A707006390070297B701009387C7E5B7
:1057B00083A7070083A7C70083A70700232EF10054
:1057C0006F008000232E01008327C101138507008D
:1057D0001301010267800000130101FD232611025D
:1057E0002326A100EFD09FA4232EA10097B701008C
:1057F000938747E283A707000327C101637CF70073
:10580000EF00C02B8327C1001307100023A0E7007F
:105810006F00C0008327C10023A0070097B70100D5
:10582000938747DF0327C10123A0E7008327C10136
:10583000138507008320C102130101036780000064
:10584000130101FD232611022326A1002324B10008
:105850002322C1002320D100232E01008327C10071
:105860000327810023A2E7008327C1000327C1008B
:1058700023A8E700032781008327410063E6E704AC
:1058800003274100832701003307F7408327C10026
:1058900083A787016368F70093071000232EF100A8
:1058A0006F00C00697B70100938747D603A707008C
:1058B0008327C100938747009385070013050700DE
:1058C000EFB08F806F008004032741008327010021
:1058D000637EF70003278100832701006368F700D8
:1058E00093071000232EF1006F00400297B70100CC
:1058F000938787D103A707008327C10093874700B9
:105900009385070013050700EFA01FFC8327C10143
:10591000138507008320C102130101036780000083
:10592000130101FD232611026F00801583278100DA
:1059300063C6071483270101232EF1008327C101C9
:1059400083A74701638A07008327C1019387470024
:1059500013850700EFB0CF8393074100138507003D
:10596000EFF09FE7232CA10083278100130790000D
:105970006368F7101397270097A701009387076CB8
:10598000B307F70003A7070097A701009387076BEA
:10599000B307F700678007000327C1008327C10111
:1059A00083A78701B307F7000327C1009306070009
:1059B00003268101938507000325C101EFF05FE80D
:1059C0001307050093071000631CF70A8327C10122
:1059D00083A747020325C101E78007008327C10190
:1059E00003A7C70193071000631CF7080327C10032
:1059F0008327C10183A78701B307F70013070000BE
:105A00009306000013860700930500000325C101DB
:105A1000EFF05FA6232AA1008327410163920706C6
:105A2000737004306F0000000327C1008327C10199
:105A300023ACE7008327C10183A787016396070092
:105A4000737004306F0000008327C10103A7870132
:105A500083278101B307F700832681010326810193
:105A6000938507000325C101EFF09FDD6F00400122
:105A70000325C101EF0090566F0080001300000065
:105A800097B701009387C7B883A707001307810062
:105A90009306000013060000930507001385070016
:105AA000EFB05F9C93070500E39207E81300000046
:105AB0008320C1021301010367800000130101FD6F
:105AC000232611026F00C00E97B701009387C7B35A
:105AD00083A7070083A7C70083A70700232CF10033
:105AE00097B70100938747B283A7070083A7C70032
:105AF00083A7C700232AF10083274101938747002A
:105B000013850700EFA0DFE88327410183A7470241
:105B100003254101E78007008327410103A7C7014F
:105B2000930710006316F7088327410183A78701B5
:105B300003278101B307F7002328F10003270101A0
:105B40008327810163F0E7048327410103270101D3
:105B500023A2E700832741010327410123A8E7008F
:105B600097B70100938747AA03A70700832741013E
:105B7000938747009385070013050700EFA0DFD444
:105B80006F00000313070000930600000326810145
:105B90009305000003254101EFF0DF8D2326A100CE
:105BA0008327C10063960700737004306F00000004
:105BB00097B70100938747A583A7070083A707002E
:105BC000E39407F097B70100938707A483A7070022
:105BD000232EF10097B70100938747A303A707007F
:105BE00097B70100938747A223A0E70097B701006A
:105BF0009387C7A10327C10123A0E700130000007A
:105C00008320C1021301010367800000130101FF1B
:105C100023261100EFE09FD897B701009387479F95
:105C200083A707006394070A17B501001305459B76
:105C3000EFA09FBA17B501001305C59BEFA0DFB910
:105C400097B701009387479C17B70100130747993F
:105C500023A0E70097B701009387479B17B7010080
:105C60001307479923A0E700130600009305C0001F
:105C700013054000EFA09FEE1307050097B7010042
:105C80009387079923A0E70097B701009387479868
:105C900083A7070063960700737004306F0000004D
:105CA00097B701009387C79683A707006380070211
:105CB00097B701009387C79583A7070097A50100B1
:105CC0009385453A13850700EFC08F9CEFE01FD105
:105CD000130000008320C100130101016780000050
:105CE000130101FD232611022326A1008327C100F1
:105CF000232EF1008327C1006396070073700430E0
:105D00006F000000EFE09FC98327C10183A747010F
:105D1000B337F00093F7F70F232CF100EFE01FCC1F
:105D200083278101138507008320C102130101032A
:105D300067800000130101FD232611022326A10024
:105D40008327C100232EF1008327C100639607003B
:105D5000737004306F000000EFE05FC48327C1015F
:105D600083A70702232CF100EFE05FC7832781019F
:105D7000138507008320C10213010103678000001F
:105D8000130101FD232611022326A1002324B100C3
:105D90008327C100232EF1008327C10063960700EB
:105DA000737004306F000000EFE05FBF8327C10114
:105DB0000327810023A0E702EFE05FC21300000089
:105DC0008320C1021301010367800000130101FE5B
:105DD000232E11001305C001EF0090002326A1001F
:105DE0008327C100638E07008327C10023A007001B
:105DF0008327C1009387470013850700EFA0DF9D2D
:105E00008327C100138507008320C101130101020C
:105E100067800000130101FC232E11022326A1003C
:105E20002324B1002322C1002320D1008327C100F5
:105E30002324F1022322010203274100B70700FFB8
:105E4000B377F70063860700737004306F000000BB
:105E50008327410063960700737004306F000000D1
:105E6000EFE05F8593070500639607008327010035
:105E700063960700930710006F00800093070000EF
:105E800063960700737004306F000000EFD0CF9A64
:105E90008327810283A707002320F1028325810045
:105EA0000325C100EF008041032701028327810001
:105EB0003367F70083274100B377F70003274100DA
:105EC000631CF7020327010283278100B367F700F1
:105ED0002326F1028327810203A7070083274100BD
:105EE00093C7F7FF3377F7008327810223A0E700EA
:105EF000232001006F00400483270100638807020C
:105F0000832781029386470003274100B7070005D6
:105F1000B367F70003260100938507001385060089
:105F2000EFD0DFA4232601026F0000018327810246
:105F300083A707002326F102EFD04F92232EA10062
:105F400083270100638407088327C1016394070046
:105F5000EFA00FE4EFE05FAE2326A1020327C1020A
:105F6000B7070002B377F70063980704EFE01FA3B9
:105F70008327810283A707002326F1020327C1029A
:105F800083274100B377F700032741006310F7022E
:105F90008327810203A707008327410093C7F7FFE8
:105FA0003377F7008327810223A0E700EFE01FA3E8
:105FB000930710002322F1020327C102B707000153
:105FC0009387F7FFB377F7002326F1028327C102F7
:105FD000138507008320C1031301010467800000BB
:105FE000130101FB23261104232EA100232CB10051
:105FF000232AC1002328D1002326E1008327C101E1
:10600000232AF102232C0102232801028327C10144
:1060100063960700737004306F000000032781014E
:10602000B70700FFB377F70063860700737004308B
:106030006F000000832781016396070073700430AE
:106040006F000000EFE00FE793070500639607007D
:106050008327C10063960700930710006F0080003C
:106060009307000063960700737004306F00000010
:10607000EFC09FFC8327410383A707002326F1027B
:1060800003260101832581010325C102EF00404B56
:106090002324A10283278102638C07028327C10284
:1060A000232EF1022326010083274101638807087C
:1060B0008327410303A707008327810193C7F7FFC5
:1060C0003377F7008327410323A0E7006F00000721
:1060D0008327C100639807008327C102232EF102A2
:1060E0006F00C00583274101638A070003278103EE
:1060F000B7070001B367F700232CF10283270101E2
:10610000638A070003278103B7070004B367F7001A
:10611000232CF10283274103938647000327810143
:1061200083278103B367F7000326C1009385070027
:1061300013850600EFD09F83232E0102EFC01FF2CC
:106140002322A1028327C100638807088327410215
:1061500063940700EFA0CFC3EFE01F8E232EA102B0
:106160000327C103B7070002B377F700639C070456
:10617000EFE0DF828327410383A70700232EF1028C
:1061800003260101832581010325C103EF00403B64
:106190009307050063840702832741016380070298
:1061A0008327410303A707008327810193C7F7FFD4
:1061B0003377F7008327410323A0E700EFE01F8236
:1061C000232801020327C103B70700019387F7FFC4
:1061D000B377F700232EF1028327C103138507004D
:1061E0008320C1041301010567800000130101FD34
:1061F000232611022326A1002324B1008327C100F6
:10620000232EF1008327C1006396070073700430CA
:106210006F00000003278100B70700FFB377F70086
:1062200063860700737004306F000000EFE00FF723
:106230008327C10183A70700232CF1008327C10115
:1062400003A707008327810093C7F7FF3377F70081
:106250008327C10123A0E700EFE04FF883278101E6
:10626000138507008320C10213010103678000002A
:10627000130101FD232611022326A1008327C1005B
:10628000232EF100EFA00FC893070500232CF10087
:106290008327C10183A70700232AF10083278101F7
:1062A00013850700EFA04FC4832741011385070022
:1062B0008320C1021301010367800000130101FB69
:1062C000232611042326A1002324B100232C01023C
:1062D0008327C1002328F102232A01028327C1005A
:1062E00063960700737004306F000000032781007D
:1062F000B70700FFB377F7006386070073700430B9
:106300006F00000083270103938747002326F102D3
:106310008327C102938787002324F102EFC0DFD1D6
:106320008327C10283A7C700232EF102832701031D
:1063300003A70700832781003367F7008327010342
:1063400023A0E7006F00000E8327C10383A7470047
:106350002322F1028327C10383A707002320F10230
:10636000232A010203270102B70700FFB377F700D2
:10637000232EF10003270102B70700019387F7FFDF
:10638000B377F7002320F1020327C101B707000408
:10639000B377F700639207028327010303A707007F
:1063A00083270102B377F700638807029307100081
:1063B000232AF1026F0040028327010303A707008D
:1063C00083270102B377F700032701026316F70062
:1063D00093071000232AF1028327410363800704F7
:1063E0000327C101B7070001B377F700638A0700ED
:1063F0000327810383270102B367F700232CF102EF
:106400008327010303A70700B7070002B367F7005C
:10641000938507000325C103EFD05F8283274102E4
:10642000232EF1020327C10383278102E31EF7F025
:106430008327010303A707008327810393C7F7FF7F
:106440003377F7008327010323A0E700EFC01FC1C4
:106450008327010383A70700138507008320C10456
:106460001301010567800000130101FD23261102BD
:106470002326A1008327C100232EF1008327C10119
:1064800093874700232CF100EFC01FBB6F00400330
:106490008327810103A7C700832781019387870092
:1064A0006316F700737004306F00000083278101CA
:1064B00083A7C700B705000213850700EFD00FF8C8
:1064C0008327810183A70700E39407FC0325C1010B
:1064D000EF00C030EFC09FB8130000008320C1025E
:1064E0001301010367800000130101FE232E110038
:1064F0002326A1002324B100832581000325C100A8
:10650000EFF0DFDB130000008320C1011301010263
:1065100067800000130101FE232E11002326A10035
:106520002324B100832581000325C100EFF01FCC97
:10653000130000008320C1011301010267800000E5
:10654000130101FE2326A1002324B1002322C10050
:10655000232E010083274100639007020327C10017
:1065600083278100B377F700638607029307100043
:10657000232EF1006F0000020327C1008327810052
:10658000B377F700032781006316F7009307100025
:10659000232EF1008327C101138507001301010297
:1065A00067800000130101FE2326A1008327C1009C
:1065B000232CF1008327C10063960700232E0100DE
:1065C0006F0000018327810183A78701232EF1003B
:1065D0008327C101138507001301010267800000B2
:1065E000130101FC232E11022326A1002322010204
:1065F000EFC09FA4973703009387070383A7070083
:10660000639C0700EF00002C973703009387C701B6
:106610001307100023A0E7008327C100638A070245
:1066200093078000138707008327C100B387E70023
:106630002326F1008327C10093F73700638A070000
:106640008327C10093F7C7FF938747002326F100F4
:106650008327C100638207160327C100B797010093
:106660009387B7FF63EAE714973703009387C7FA66
:106670002324F10297370300938707FA83A70700C3
:106680002326F1026F0080018327C1022324F10237
:106690008327C10283A707002326F1028327C102B3
:1066A00083A747000327C10063F8E7008327C102DF
:1066B00083A70700E39A07FC0327C102973703006B
:1066C000938707F6630AF70E8327810283A70700E3
:1066D00013078000B387E7002322F1028327C1025A
:1066E00003A707008327810223A0E7008327C102B5
:1066F00003A747008327C100B307F74013078000B3
:10670000131717006378F7080327C1028327C10016
:10671000B307F700232EF1008327C10203A7470028
:106720008327C1003307F7408327C10123A2E70075
:106730008327C1020327C10023A2E7008327C101E9
:1067400083A74700232CF100973703009387C7ECFA
:106750002320F1026F0000018327010283A70700B5
:106760002320F1028327010283A7070083A74700A4
:1067700003278101E3E2E7FE8327010203A7070065
:106780008327C10123A0E700832701020327C1015A
:1067900023A0E70097A70100938747C503A7070039
:1067A0008327C10283A747003307F74097A701005B
:1067B0009387C7C323A0E700EFC05F8A8327410206
:1067C00063940700EF10801F8327410213850700A1
:1067D0008320C1031301010467800000130101FD40
:1067E000232611022326A1008327C100232CF100B8
:1067F0008327C1006382070A93078000B307F04034
:1068000003278101B307F700232CF10083278101BF
:10681000232AF100EFC05F828327410183A747004D
:106820002328F10097370300938707DF232EF10019
:106830006F0000018327C10183A70700232EF10009
:106840008327C10183A7070083A74700032701010E
:10685000E3E2E7FE8327C10103A707008327410185
:1068600023A0E7008327C1010327410123A0E700FC
:106870008327410103A7470097A70100938707B724
:1068800083A707003307F70097A70100938707B690
:1068900023A0E700EFC08FFC130000008320C1029B
:1068A000130101036780000097A70100938707B4D5
:1068B00083A707001385070067800000130000000E
:1068C00067800000130101FF97A70100938707D598
:1068D00093F7C7FF2326F100973703009387C7D3A9
:1068E0000327C10023A0E700973703009387C7D28F
:1068F00023A2070097370300938787D237970100B9
:106900001307C7FF23A2E70097370300938747D1F8
:1069100023A007008327C1002324F10083278100DF
:10692000379701001307C7FF23A2E70083278100E1
:10693000173703001307C7CE23A0E700130000009A
:106940001301010167800000130101FE2326A1004D
:106950002324B1002322C10083278100232EF100CC
:106960008327C100232CF1000327C1008327810066
:10697000B367F70093F73700639607066F00C0020E
:106980008327C10103A707008327810123A0E70014
:106990008327810193874700232CF1008327C101BE
:1069A00093874700232EF100832741009387D7FF69
:1069B0000327C100B307F70003278101E362F7FC57
:1069C0006F0040020327C10193071700232EF10037
:1069D0008327810193861700232CD10003470700EA
:1069E0002380E7000327C10083274100B307F70096
:1069F00003278101E368F7FC8327C10013850700A3
:106A00001301010267800000130101FE2326A1008B
:106A10002324B1002322C1000327C10083274100A2
:106A2000B367F70093F73700639807068327810061
:106A300093F7F70F232AF1008327410193978700EB
:106A400003274101B367F700232AF100832741019F
:106A50009397070103274101B367F700232AF10049
:106A60008327C100232EF1006F0080018327C1011D
:106A700013874700232EE1000327410123A0E700ED
:106A80000327C10083274100B307F7000327C10193
:106A9000E36EF7FC6F00C0038327C100232CF100D5
:106AA0006F00C0018327810113871700232CE100A9
:106AB000032781001377F70F2380E7000327C10026
:106AC00083274100B307F70003278101E36CF7FC3C
:106AD0008327C100138507001301010267800000AE
:106AE000130101FE2326A1008327C100232EF100FC
:106AF0006F0000018327C10193871700232EF10047
:106B00008327C10183C70700E39607FE0327C1015E
:106B10008327C100B307F740138507001301010263
:106B200067800000130101FE2326A1002324B10089
:106B30008327C100138717002326E10083C70700BE
:106B4000A30FF10083278100138717002324E1009E
:106B500083C70700230FF1008347F1016388070013
:106B60000347F1018347E101E304F7FC0347F10127
:106B70008347E101B307F7401385070013010102C2
:106B800067800000130101FE2326A1002324B10029
:106B90008327C100232EF10013000000032781008A
:106BA000930717002324F1008327C1019386170060
:106BB000232ED100034707002380E70083C7070087
:106BC000E39E07FC8327C100138507001301010220
:106BD00067800000130101FE2326A100232E01007F
:106BE000232C01006F0000018327C1009387170049
:106BF0002326F1008327C10003C707009307000283
:106C0000E304F7FE8327C10003C707009307D00200
:106C1000630AF7008327C10003C707009307B00288
:106C20006312F7068327C10083C70700938737FDE8
:106C300093B7170093F7F70F232CF1008327C100B8
:106C4000938717002326F1006F00C0030327C101BB
:106C50009307070093972700B387E70093971700E0
:106C6000232EF1008327C100138717002326E1009C
:106C700083C70700938707FD0327C101B307F70008
:106C8000232EF1008327C10083C70700E39007FC90
:106C900083278101638807008327C101B307F04080
:106CA0006F0080008327C1011385070013010102D3
:106CB00067800000130101FE2326A100973703001F
:106CC0009387479883A70700938617001737030019
:106CD000130747972320D7000327C1001377F70F27
:106CE000973603009386069AB387F6002380E70061
:106CF0000327C1009307A000630CF7009737030038
:106D00009387479403A7070093070004631EF704C3
:106D10009737030093870797232EF1006F00C00376
:106D20008327C10113871700232EE10003C7070043
:106D3000B70710F0938707F023A0E7009737030009
:106D40009387479083A707001387F7FF97370300C0
:106D50009387478F23A0E700973703009387878E99
:106D600083A70700E39E07FA930700001385070037
:106D70001301010267800000130101EB23261114A7
:106D8000232481142322911423202115232E31132F
:106D9000232C4113232A5113232EA100232CB100AD
:106DA0002328C100232AD1002326E1002324F10057
:106DB00023220101232601128327C100138A070021
:106DC000930A0000832701010328410113060A00EA
:106DD00093860A001385070093050800EF10105CE6
:106DE0009307050013880500138607009306080023
:106DF0008327C112138717002326E1121307060009
:106E00009397270093060113B387F60023AEE7EEAE
:106E10008327C100138407009304000083274101E6
:106E20001387040063E8E704832741011387040004
:106E30006398E700832701011307040063ECE7026E
:106E40008327C10013890700930900001306090076
:106E5000938609000325010183254101EF10407647
:106E600093070500138805002328F100232A010158
:106E70006FF09FF4130000006F0040018327C101F1
:106E80008325810103254100E780070083278100D6
:106E90001387F7FF2324E1000327C112E340F7FE25
:106EA0006F0040058327C112939727001307011332
:106EB000B307F70003A7C7EF8327C11293972700F3
:106EC00093060113B387F60083A6C7EF93079000DC
:106ED00063F6D700930770056F00800093070003E7
:106EE000B387E7000327C1018325810113850700CC
:106EF000E70007008327C1121387F7FF2326E1125B
:106F0000E342F0FA130000008320C114032481142B
:106F100083244114032901148329C113032A8113F3
:106F2000832A41131301011567800000130101FF3B
:106F30002326A1002324B10083268100130710001B
:106F40006356D7028327C10083A707009387770082
:106F500093F787FF938687000327C1002320D7007C
:106F600003A8470083A707006F00000503278100DF
:106F7000630407020327C100032707001306470025
:106F80008326C10023A0C60003270700930707003C
:106F9000130800006F0040020327C1000327070009
:106FA000130647008326C10023A0C600032707005D
:106FB00093070700130800001385070093050800D6
:106FC0001301010167800000130101FF2326A100C6
:106FD0002324B10083268100130710006356D702D3
:106FE0008327C10083A707009387770093F787FF64
:106FF000938687000327C1002320D70003A84700FA
:1070000083A707006F00800503278100630607023E
:107010000327C10003270700130647008326C1008A
:1070200023A0C60003270700930707001357F74163
:10703000130807006F0080020327C1000327070021
:10704000130647008326C10023A0C60003270700BC
:10705000930707001357F74113080700138507002C
:10706000930508001301010167800000130101FC72
:10707000232E1102232C8102232A91022326A10010
:107080002324B1002322C1002320D1006F0040023D
:107090006300043C83274100938717002322F100FB
:1070A0008327C1008325810013050400E7800700C2
:1070B0008327410083C7070013840700930750020A
:1070C000E318F4FC83274100938717002322F10083
:1070D000832741002328F10093070002A30BF1004E
:1070E0009307F0FF232EF1009307F0FF232CF1000C
:1070F0002320010283274100138717002322E10088
:1071000083C70700138407009307D4FD13075005B6
:107110006360F7321397270097970100938787F5ED
:10712000B307F70003A7070097970100938787F439
:10713000B307F700678007009307D002A30BF100A5
:107140006FF05FFB93070003A30BF1006FF09FFA52
:10715000232C010003278101930707009397270041
:10716000B387E70093971700B307F400938707FDF1
:10717000232CF1008327410083C7070013840700F5
:107180009307F00263D287049307900363CE8702CC
:1071900083274100938717002322F1006FF09FFBA4
:1071A00083270100138747002320E10083A70700FE
:1071B000232CF1006F0080018327C101E3DC07F27B
:1071C000232E01006FF01FF3130000008327C1017D
:1071D000E3D207F283278101232EF1009307F0FF0A
:1071E000232CF1006FF01FF1832701029387170012
:1071F0002320F1026FF01FF083270100138747005F
:107200002320E10083A707000327C1008325810015
:1072100013850700E70007006F0040238327010064
:10722000138747002320E10083A40700639604002E
:1072300097940100938484E38327C1016350F0088D
:10724000034771019307D002630AF7068327810180
:107250009385070013850400EF10403413070500E1
:107260008327C101B387E740232EF1006F0040025E
:10727000834771010327C10083258100138507001F
:10728000E70007008327C1019387F7FF232EF10052
:107290008327C101E34EF0FC6F0040028327C10049
:1072A0008325810013050400E78007009384140000
:1072B0008327C1019387F7FF232EF10083C70400C2
:1072C000138407006300040483278101E3C807FCDB
:1072D000832781019387F7FF232CF1008327810106
:1072E000E3DE07FA6F0000028327C10083258100D7
:1072F00013050002E78007008327C1019387F7FF8A
:10730000232EF1008327C101E340F0FE6F0000143B
:10731000930701008325010213850700EFF0DFCA00
:1073200093070500138805002324F1022326010397
:10733000832781020328C1029307080063D607044C
:107340008327C100832581001305D002E780070051
:10735000832581020326C102930700001308000061
:10736000B386B7401385060033B5A7003307C8407E
:10737000B307A74013870700938706001308070089
:107380002324F102232601039307A0002322F10204
:107390006F0040069307A0002322F1026F00000453
:1073A000930780002322F1026F004003930710002F
:1073B0002320F1028327C1008325810013050003E8
:1073C000E78007008327C10083258100130580071C
:1073D000E7800700930700012322F10293070100D1
:1073E0008325010213850700EFF05FB42324A10277
:1073F0002326B10203274102834771011388070046
:107400008327C101032681028326C10283258100CF
:107410000325C100EFF05F966F0040038327C10092
:107420008325810013050400E78007006F00000238
:107430008327C1008325810013055002E7800700E0
:10744000832701012322F100130000006FF05FC6C3
:10745000130000008320C10303248103832441031C
:107460001301010467800000130101FF2326A1001E
:10747000B70710F0938707F20327C10023A0E700A6
:107480006F000000130101FB232611022326A10037
:10749000232AB102232CC102232ED1022320E1048E
:1074A0002322F10423240105232611059307010556
:1074B000938747FE232EF1008327C101938607009F
:1074C0000326C1009305000017F5FFFF1305C57ED5
:1074D000EFF0DFB993070000138507008320C10296
:1074E0001301010567800000130101FE2326A1009E
:1074F0002324B1002322710083278100232EF10071
:107500008327C10183A707000327C1001377F70F63
:107510002380E7008327C10183A707001387170093
:107520008327C10123A0E70013000000130101021B
:1075300067800000130101FA232E11022326A10007
:107540002324B1002324C1042326D1042328E104E9
:10755000232AF104232C0105232E1105930701068C
:107560002322F10293074101930541011706000010
:107570001306C6F737F7FFFF9346F7FF37150000EE
:10758000130505803388A5003378E8001368783B3D
:1075900023A007013305A6003377E500136777338F
:1075A00023A2E70033F7D50093154701378703007F
:1075B0001307373933E7E50023A4E7003377D60014
:1075C00093164701370703001307770633E7E600F2
:1075D00023A6E7000F1000008327C1002326F10235
:1075E00093070106938787FE2324F1020327810274
:1075F00093074101138507009307C1009306070015
:107600000326810093850700EFF05FA68327C10062
:10761000238007008327C100138707008327C10247
:10762000B307F740138507008320C1031301010648
:1076300067800000130101FF370510F0130545F4C2
:10764000032505002326A100370510F0130505F4D6
:10765000032505002324A100370510F0130545F488
:10766000032505008328C100E398A8FC0325C10079
:107670001303050093030000131703009306000093
:10768000032581009305050013060000B3E7B6004B
:107690003368C700370710F0130587F4B7150000EB
:1076A000938505FA13060000B386B7009388060099
:1076B000B3B8F8003307C800B387E80013870700A2
:1076C00093870600130807002320F50023220501F5
:1076D000130000001301010167800000130101FF86
:1076E00023261100EFF01FF59307000873A0473021
:1076F000130000008320C100130101016780000016
:10770000130101FE232E11002326A100179501006D
:107710001305C5ABEFF01FD7130000008320C10194
:107720001301010267800000130101FE232E1100E6
:107730002326A100179501001305C5A9EFF09FD4DA
:10774000130000008320C1011301010267800000C3
:10775000130101FD232611022326A100232E01007F
:107760006F004001130000008327C10193871700B9
:10777000232EF1000327C101B71700009387773844
:10778000E3D2E7FE17950100130545A5EFF09FCF63
:107790006FF0DFFC130101FD232611022326A10057
:1077A000232E01006F004001EF00C06D8327C1014F
:1077B00093871700232EF1000327C101930730019F
:1077C000E3D4E7FE130000008320C102130101038C
:1077D00067800000130101FE232E1100EF004020FE
:1077E00017070000130747FB93060000130610005D
:1077F00093052003179501001305C59EEFD05FBCCC
:107800002326A100EFB09FA29307050013070000F5
:107810009306000013860700930510000325C1009E
:10782000EFD05FC5130000008320C10113010102E6
:1078300067800000130101FE232E110023260100A2
:10784000EF0040231307050093071000630EF700B5
:107850001795010013058599EFF0DFC28327C1005A
:1078600093E727002326F1008327C1001385070033
:107870008320C1011301010267800000130101FE92
:10788000232E110023260100EFF0DFF4170700007C
:1078900013078706930600001306100093054006A1
:1078A0001795010013050596EFD09FB12326A1007F
:1078B0008327C10063820702EFB05F97930705003B
:1078C00013070000930600001386070093051000BD
:1078D0000325C100EFD01FBA23240100EFB00FE849
:1078E00093070000138507008320C10113010102E3
:1078F00067800000130101FD232611022326A10049
:1079000097970100938787AD83A7070013874706E2
:1079100097970100938787AC23A0E7009797010012
:10792000938707AC83A70700138747069797010043
:10793000938707AB23A0E70097970100938707AAD7
:1079400003A707009307F07C63DEE7049797010025
:107950009387C7A883A7070013870783979701001A
:107960009387C7A723A0E700EFF0DFEC232EA10049
:107970008327C101639E070097970100938747A65D
:1079800003A70700B71700009387F77663D0E702D5
:107990008327C10113850700EFF01FADEFB00FE79C
:1079A0006F000001130000006F0080001300000052
:1079B0008320C1021301010367800000737004304B
:1079C0006F0000001300000067800000130101FF3A
:1079D0002326A1002324B100737004306F0000003F
:1079E000130101FF23261100930800001308000073
:1079F00097270300938707D613071000930600000C
:107A000013060040979501009385858017050000B7
:107A100013058519EFA01F8797270300938787D346
:107A200083A60700930800001308000097270300AF
:107A3000938787D213071000130600409785010033
:107A40009385857D170500001305C535EFA09F833D
:107A500097270300938707D083A7070013850700A4
:107A6000EFB04F92130000008320C1001301010109
:107A700067800000130101FF930710002326F10027
:107A800097270300938787C603A70700972703005C
:107A9000938707C583A707006314F7002326010017
:107AA000972703009387C7C303A7070097270300FF
:107AB0009387C7C323A0E700232401006F0080073A
:107AC000172703001307C7C2832781009397270056
:107AD000B307F70003A7070097260300938646BF66
:107AE0008327810093972700B387F60083A70700B9
:107AF0006314F7002326010017270300130747BD6F
:107B00008327810093972700B307F70003A7070097
:107B1000972603009386C6BD83278100939727008D
:107B2000B387F60023A0E70083278100938717001F
:107B30002324F1000327810093072000E3D2E7F814
:107B4000979701009387078B03A7070093071000FF
:107B50006304F70023260100979701009387C789E4
:107B600003A7070097270300938747B983A7070058
:107B70006316F700232601006F00C00197970100EC
:107B80009387878703A7070097270300938707B783
:107B900023A0E7008327C10013850700130101011B
:107BA00067800000130101FD232611022326A10096
:107BB000232A01009307410113850700EF00D01B22
:107BC000EF0090149307050093053000138507001C
:107BD000EF10005493070500232EF1001727030030
:107BE000130747AE8327C10193972700B307F70018
:107BF00083A70700232CF10017270300130747ADC5
:107C00008327C10193972700B307F70083A70700D5
:107C10001387170097260300938686AB8327C1013D
:107C200093972700B387F60023A0E700930741014D
:107C3000930600001306F0FF9385070003258101DA
:107C4000EF904FAB13070500930710006308F70090
:107C5000978701009387077A23A0070083274101B4
:107C600093871700232AF10003274101B70701007A
:107C70009387F7FF6314F700232A0100EF008000C9
:107C80006FF01FF4130101FF232611009727030053
:107C9000938707A783A70700138717009727030079
:107CA000938707A623A0E70097270300938747A59C
:107CB00003A707009307100163FCE70C9727030055
:107CC000938707A423A0070097270300938787A320
:107CD00083A70700130710006382E704130710004F
:107CE00063E8E70013072000638CE7066F00400A93
:107CF00097270300938747A683A7070093050000F3
:107D000013850700EFA0DFC7972703009387879F9E
:107D10001307100023A0E7006F00800797270300D8
:107D2000938787A383A70700930510001385070097
:107D3000EFA01FC5972703009387C7A183A707005C
:107D40009305000013850700EFA09FC3972703004A
:107D50009387479B1307200023A0E7006F00400391
:107D6000972703009387079F83A7070093051000B9
:107D700013850700EFA0DFC097270300938787983C
:107D800023A007001305800CEFA0DF9B1300000069
:107D9000130000008320C10013010101678000006F
:107DA000130101FD232611022326A100EF00404B01
:107DB00013050000EFA05FB193070500639607006D
:107DC000232E01006F00C0009307F0FF232EF10067
:107DD000972703009387879083A707009305F0FFF9
:107DE00013850700EFA08FB4232CA1008327810106
:107DF000639E07008327C101E38C07FA9787010080
:107E00009387475F23A007006FF09FFA9307410114
:107E100093060000130600009385070003258101E7
:107E2000EF904FE413070500930710006308F70075
:107E3000978701009387075C23A00700EFC01FB658
:107E40008327410113850700EF00C00AEFC01FB967
:107E5000978701009387075A03A70700930710002D
:107E6000E318F7F4972703009387878783A7070012
:107E700013871700972703009387878623A0E700BF
:107E80006FF01FF3130101FF232611009727030052
:107E90009387478503A70700930710006314F7042F
:107EA000972703009387478683A707001387170048
:107EB000972703009387478523A0E70097270300B0
:107EC0009387878403A707009307400663FCE700B6
:107ED000972703009387478323A00700EF00C02361
:107EE000EF00802A130000008320C100130101016C
:107EF00067800000130101FE232E11002326A1003C
:107F00000327C100B70701009387E7FF63FAE70A79
:107F10000327C100B707FFFF938717003307F70058
:107F20009307500063F0E7040327C100930780FF25
:107F300063EAE702978701009387474C83A707000E
:107F4000938507000325C100EF00401313070500C8
:107F5000930710006308F70097870100938787490C
:107F600023A00700978701009387C74883A70700CE
:107F700063960700737004306F000000978701005C
:107F80009387C74783A707001387170097870100C8
:107F90009387C74623A0E70097870100938707468A
:107FA00083A707006394070C978701009387074511
:107FB000370701001307F7FF23A0E7006F00000B4E
:107FC0000327C1009307500063F6E704B7070100D9
:107FD0001387E7FF8327C1003307F740930760004B
:107FE00063FAE702971703009387477283A7070096
:107FF000938507000325C100EF0040081307050023
:10800000930710006308F700978701009387873E66
:1080100023A00700978701009387C73D83A7070028
:1080200063960700737004306F0000009717030019
:108030009387C76D83A7070013871700971703005F
:108040009387C76C23A0E700971703009387076CFB
:1080500003A70700B70701009387E7FF63F8E7006E
:10806000971703009387876A23A007001300000077
:108070008320C1011301010267800000130101FE8A
:108080002326A1002324B10093071000232EF10022
:108090000327C1008327810063FEE7020327C10095
:1080A000832781003307F7409307300063F6E7002A
:1080B000737004306F0000000327C1008327810024
:1080C0003307F7409307300063F0E704232E0100E5
:1080D0006F008003032781008327C1003307F74027
:1080E0009307300063F6E700737004306F00000000
:1080F000032781008327C1003307F740930730002F
:1081000063F4E700232E01008327C10113850700D4
:108110001301010267800000130101FE232E1100EC
:10812000971703009387875B83A7070013850700D2
:10813000EFA0CF832326A1008327C100638E07020F
:108140009307810013060000938507000325C100F3
:10815000EF904FD913070500930710006308F7004D
:10816000978701009387072923A0070083278100B1
:1081700013850700EFF01FD8130000008320C10112
:108180001301010267800000130101FF2326110083
:10819000971703009387C75783A707001717030094
:1081A0001307475293972700B307F70083A70700E9
:1081B0009306000013060000978501009385C523F0
:1081C00013850700EF80DFF9130705009307100000
:1081D0006310F708978701009387072283A707009A
:1081E00013871700978701009387072123A0E700D3
:1081F000978701009387472083A70700639C0700A8
:10820000978701009387471F370701001307F7FF80
:1082100023A0E700971703009387874F83A70700E2
:1082200013871700971703009387874E23A0E70053
:10823000971703009387C74D03A7070093072000F4
:1082400063D8E700971703009387874C23A00700A4
:10825000130000008320C1001301010167800000AA
:10826000130101FE232E11002324010013059000A9
:10827000EF901FDB1307050097170300938707464E
:1082800023A0E700232601006F00000F1306000063
:108290009305400013053000EF805F8C93060500C6
:1082A00017170300130707428327C100939727007E
:1082B000B307F70023A0D700171703001307874061
:1082C0008327C10093972700B307F70083A7070010
:1082D00063960700737004306F00000017170300E7
:1082E0001307473E8327C10093972700B307F70082
:1082F00003A70700971703009387473E83A707004C
:108300009385070013050700EF90DFD413070500DE
:1083100093071000630AF700978701009387870D82
:1083200023A007006F008004171703001307873985
:108330008327C10093972700B307F70003A707001F
:10834000971703009387873983A707009385070052
:1083500013050700EF901FD09307050063880700FF
:10836000978701009387070923A007008327C1008F
:10837000938717002326F1000327C10093072000ED
:10838000E3D6E7F0971703009387C73383A7070067
:108390009305000013850700EF905FD29307050057
:1083A00063880700978701009387C70423A007000D
:1083B000971703009387073103A707009717030058
:1083C0009387C73183A7070093850700130507002C
:1083D000EF90DFCE13070500930710006308F70046
:1083E000978701009387070123A0070097170300D1
:1083F0009387472D83A7070013078100930600008A
:10840000130600009305070013850700EF809FAE59
:10841000971703009387072B03A7070097170300FD
:108420009387C72B83A707009385070013050700D1
:10843000EF905FC2930705006388070097870100EC
:10844000938747FB23A0070097170300938787278D
:1084500083A707001307810093060000130600009E
:108460009305070013850700EF80DFFF97170300D0
:108470009387472503A707009717030093870726CD
:1084800083A707009385070013050700EF909FBCA3
:1084900013070500930710006308F7009787010092
:1084A000938747F523A007009717030093870723B7
:1084B00083A707009305800C13850700EF901FC763
:1084C000930705006388070097870100938787F269
:1084D00023A00700971703009387C72783A70700E8
:1084E00013850700EFA0DF84971703009387871F8A
:1084F0001307100023A0E700130000008320C10130
:108500001301010267800000130101FF23261100FF
:10851000971703009387471D03A70700B757C64166
:108520009385D7E613050700EF0050379307050042
:1085300013870700B7370000938797033307F700C7
:10854000971703009387471A23A0E70097170300A4
:108550009387871983A7070013D70701B787000000
:108560009387F7FFB377F700138507008320C100D7
:108570001301010167800000130101FF2326A10000
:1085800097170300938747160327C10023A0E7002E
:10859000130000001301010167800000B305B5005E
:1085A000930705006386B70003C70700631607003B
:1085B0003385A74067800000938717006FF09FFE08
:1085C000130101FD23229102232A510123261102C6
:1085D0002324810223202103232E3101232C410156
:1085E0002328610123267101232481012322910183
:1085F0002320A101930A050093840500639E063899
:10860000130406009309050017890100130949C1E5
:1086100063F8C512B7070100138B05006378F610E5
:108620001307F00F3337C70013173700B357E600AF
:108630003309F900834609003387E60093060002F8
:10864000B386E640638C0600B394D40033D7EA00C7
:108650003314D600336B9700B399DA00935A0401B0
:1086600093850A0013050B00EF00902A13090500FB
:1086700093850A00931B040113050B00EF00D0241F
:1086800093DB0B01930405009305050013850B0094
:10869000EF00D0201319090193D70901B367F9003E
:1086A000138A040063FEA700B3878700138AF4FFD0
:1086B00063E8870063F6A700138AE4FFB3878700A7
:1086C000B384A74093850A0013850400EF0050246B
:1086D0001309050093850A0013850400EF00D01EDE
:1086E00093990901930405009305050013190901E5
:1086F00013850B0093D90901EF00501AB3693901B2
:108700001386040063FCA900B30934011386F4FF47
:1087100063E6890063F4A9001386E4FF13140A01D9
:108720003364C400130A00006F000013B707000190
:1087300013070001E36CF6EE130780016FF01FEFE3
:10874000138A0600631A0600930500001305100043
:10875000EF00901713040500B7070100637EF412C1
:108760009307F00F63F48700130A8000B3574401A6
:108770003309F90003470900930600023307470154
:10878000B386E64063940612B3848440130A100053
:10879000135B040193050B0013850400EF005017D1
:1087A0001309050093050B0013850400931B0401B6
:1087B000EF00901193DB0B01930405009305050076
:1087C00013850B00EF00900D1319090193D70901D0
:1087D000B367F900938A040063FEA700B38787009C
:1087E000938AF4FF63E8870063F6A700938AE4FFA7
:1087F000B3878700B384A74093050B00138504005B
:10880000EF0010111309050093050B0013850400F8
:10881000EF00900B9399090193040500930505005F
:108820001319090113850B0093D90901EF001007F3
:10883000B36939011386040063FCA900B30934014C
:108840001386F4FF63E6890063F4A9001386E4FF4E
:1088500013940A013364C4001305040093050A004D
:108860008320C102032481028324410203290102DF
:108870008329C101032A8101832A4101032B0101BC
:10888000832BC100032C8100832C4100032D0100A8
:108890001301010367800000B7070001130A0001FC
:1088A000E366F4EC130A80016FF05FEC3314D4003C
:1088B00033DAE400B399DA0033D7EA00935A0401BB
:1088C000B394D40093850A0013050A00336B970014
:1088D000EF0010041309050093850A0013050A0030
:1088E000931B0401EF00407E93DB0B019304050012
:1088F0009305050013850B00EF00407A1319090159
:1089000013570B013367E900138A0400637EA70045
:1089100033078700138AF4FF636887006376A70034
:10892000138AE4FF33078700B304A74093850A0046
:1089300013850400EF00C07D1309050093850A002C
:1089400013850400EF0040789304050093050500AB
:1089500013850B00EF00807413170B0113570701E9
:1089600013190901B367E9001387040063FEA70028
:10897000B38787001387F4FF63E8870063F6A700D7
:108980001387E4FFB3878700131A0A01B384A74053
:10899000336AEA006FF0DFDF63ECD51EB707010032
:1089A00063F4F6041307F00FB335D7009395350041
:1089B00033D7B6009787010093878786B387E70090
:1089C00003C70700130A00023307B700330AEA405F
:1089D00063160A0213041000E3E096E833B6CA00F7
:1089E000134416006FF05FE7B7070001930500011D
:1089F000E3E0F6FC930580016FF09FFBB35CE600BB
:108A0000B3964601B3ECDC0033D4E40093DB0C01F5
:108A1000B397440133D7EA0093850B001305040094
:108A2000336BF700B3194601EF00806E13090500A0
:108A300093850B0013050400139C0C01EF00C06824
:108A4000135C0C01930405009305050013050C004D
:108A5000EF00C0641319090113570B013367E900D4
:108A600013840400637EA700330797011384F4FF87
:108A7000636897016376A7001384E4FF33079701C7
:108A8000B304A74093850B0013850400EF004068F2
:108A90001309050093850B0013850400EF00C062E5
:108AA000930405009305050013050C00EF00005F1B
:108AB00093170B011319090193D70701B367F90045
:108AC0001386040063FEA700B38797011386F4FFA3
:108AD00063E8970163F6A7001386E4FFB387970165
:108AE00013140401B70B01003364C4001389FBFFA6
:108AF000337D240133F92901B384A740930509008C
:108B000013050D00EF008059935C040193050900E3
:108B1000130B050013850C00EF00405893D9090191
:108B2000130C05009385090013850C00EF00005716
:108B3000130905009385090013050D00EF00005689
:108B40003305850193570B013385A70063748501B5
:108B50003309790193570501B387270163E6F402CE
:108B6000E392F4BCB70701009387F7FF3375F50074
:108B700013150501337BFB0033964A01330565016C
:108B8000130A0000E37AA6CC1304F4FF6FF09FB938
:108B9000130A0000130400006FF01FCC130101FB47
:108BA0002324810423229104232E310323229103C1
:108BB0002326110423202105232C4103232A5103BA
:108BC0002328610323267103232481032320A10387
:108BD000232EB101930C05009389050013040500B1
:108BE00093840500639E062613090600138A060077
:108BF000977A0100938ACA6263F4C514B70701002B
:108C00006376F6129307F00F63F4C700130A80002F
:108C1000B3574601B38AFA0003C70A0013050002DE
:108C200033074701330AE540630C0A00B395490155
:108C300033D7EC0033194601B364B70033944C01C9
:108C4000935A090193850A0013850400EF00404CF4
:108C50009309050093850A00131B0901138504007D
:108C6000EF008046135B0B019305050013050B0015
:108C7000EF00C0429399090193570401B3E7F9004B
:108C800063FAA700B387270163E6270163F4A7000F
:108C9000B3872701B384A74093850A001385040096
:108CA000EF0000479309050093850A00138504002F
:108CB000EF00804113140401930505009399090105
:108CC00013050B0013540401EF00403D33E4890009
:108CD000637AA40033042401636624016374A4004E
:108CE000330424013304A4403355440193050000A8
:108CF0008320C10403248104832441040329010443
:108D00008329C103032A8103832A4103032B01031F
:108D1000832BC102032C8102832C4102032D01020B
:108D2000832DC1011301010567800000B707000111
:108D3000130A0001E36EF6EC130A80016FF05FED99
:108D4000631A06009305000013051000EF00C037FA
:108D500013090500B7070100637AF90E9307F00FB6
:108D600063F42701130A8000B3574901B38AFA005C
:108D700003C70A0013050002B384294133074701E2
:108D8000330AE540E30E0AEA33194901B3DAE90090
:108D9000B395490133D7EC0093540901336BB70005
:108DA00013850A0093850400EF00803693090500BF
:108DB00093850400931B090113850A00EF00C0305E
:108DC00093DB0B019305050013850B00EF00002DCD
:108DD0009399090193570B01B3E7F90033944C01C0
:108DE00063FAA700B387270163E6270163F4A700AE
:108DF000B3872701B38AA7409385040013850A002F
:108E0000EF000031930905009385040013850A00E3
:108E1000EF00802B9305050013850B00EF00002861
:108E200093150B019399090193D50501B3E5B90099
:108E300063FAA500B385250163E6250163F4A50067
:108E4000B3852501B384A5406FF09FDFB70700010C
:108E5000130A0001E36AF9F0130A80016FF0DFF0F2
:108E6000E3E8D5E8B707010063FCF604930BF00FC5
:108E700033B5DB001315350033D7A6009777010013
:108E80009387073AB387E70083CB07009305000277
:108E9000B38BAB00338B7541631E0B0263E4360169
:108EA00063EACC003384CC40B386D94033B58C0020
:108EB000B384A64013050400938504006FF05FE3BC
:108EC000B707000113050001E3E8F6FA1305800176
:108ED0006FF09FFAB3966601335D7601336DDD0066
:108EE00033D47901B395690133DC7C0193540D01CE
:108EF000336CBC001305040093850400B31A6601AB
:108F0000EF000021130A05009385040013050400F7
:108F100033996C01931C0D01EF00001B93DC0C01D5
:108F2000130405009305050013850C00EF000017DE
:108F3000131A0A0113570C013367EA00130A0400DD
:108F4000637EA7003307A701130AF4FF6368A70134
:108F50006376A700130AE4FF3307A701B309A7400C
:108F60009385040013850900EF00801A938504009F
:108F70001304050013850900EF0000159305050093
:108F80009304050013850C00EF00401193150C01AC
:108F90001314040193D50501B365B40013870400CD
:108FA00063FEA500B385A5011387F4FF63E8A5015F
:108FB00063F6A5001387E4FFB385A501131A0A0120
:108FC000B70C0100336AEA001384FCFFB3778A0010
:108FD00033F48A00B384A540138507009305040089
:108FE0002326F100135A0A01EF00400B93090500F4
:108FF0009305040013050A00EF00400A13DC0A0180
:10900000930D050093050C0013050A00EF000009FD
:109010008327C100130A050093050C001385070080
:10902000EF00C0073305B50113D709013307A700C7
:109030006374B701330A9A01B70701009387F7FFFA
:10904000935507013377F70013170701B3F7F900BA
:10905000B3854501B307F70063E6B400639EB4002F
:10906000637CF90033865741B3B7C700B385A54188
:10907000B385F54093070600B307F9403339F9008B
:10908000B385B440B385254133947501B3D76701E7
:109090003365F400B3D565016FF09FC51306050075
:1090A0001305000093F61500638406003305C50020
:1090B00093D5150013161600E39605FE6780000091
:1090C0006340050663C60506138605009305050083
:1090D0001305F0FF630C060293061000637AB600D6
:1090E0006358C0001316160093961600E36AB6FE86
:1090F0001305000063E6C500B385C5403365D500A0
:1091000093D6160013561600E39606FE67800000FD
:1091100093820000EFF05FFB13850500678002007B
:109120003305A04063D80500B305B0406FF0DFF908
:10913000B305B04093820000EFF01FF93305A04063
:10914000678002009382000063CA0500634C05003B
:10915000EFF09FF71385050067800200B305B0406C
:10916000E35805FE3305A040EFF01FF63305B0408D
:049170006780020012
:02000004800278
:1000000049444C4500000000684EFEFF004EFEFFD4
:100010001C4EFEFF344EFEFF444EFEFF3850FEFFE6
:10002000D04FFEFFEC4FFEFF0450FEFF1450FEFFCA
:10003000546D7220537663006059FEFF6059FEFFD5
:100040006059FEFF485AFEFFF059FEFF385AFEFF86
:100050006059FEFF6059FEFF485AFEFFF059FEFF4F
:10006000546D725100000000286E756C6C29000000
:100070008470FEFFC073FEFFAC73FEFFC073FEFF13
:10008000C073FEFFC073FEFFC073FEFF3071FEFF42
:10009000C073FEFFC073FEFFC870FEFF4871FEFF15
:1000A000C073FEFFD470FEFFE070FEFFE070FEFF45
:1000B000E070FEFFE070FEFFE070FEFFE070FEFF0C
:1000C000E070FEFFE070FEFFE070FEFFC073FEFF19
:1000D000C073FEFFC073FEFFC073FEFFC073FEFF60
:1000E000C073FEFFC073FEFFC073FEFFC073FEFF50
:1000F000C073FEFFC073FEFFC073FEFFC073FEFF40
:10010000C073FEFFC073FEFFC073FEFFC073FEFF2F
:10011000C073FEFFC073FEFFC073FEFFC073FEFF1F
:10012000C073FEFFC073FEFFC073FEFFC073FEFF0F
:10013000C073FEFFC073FEFFC073FEFFC073FEFFFF
:10014000C073FEFFC073FEFFC073FEFFC073FEFFEF
:10015000C073FEFFC073FEFFC073FEFFC073FEFFDF
:10016000C073FEFFC073FEFFC073FEFFC073FEFFCF
:100170008871FEFFA072FEFFC073FEFFC073FEFF1A
:10018000C073FEFFC073FEFFC073FEFFC073FEFFAF
:10019000C073FEFF7871FEFFC073FEFFC073FEFFE9
:1001A0003073FEFF3C73FEFFC073FEFFC073FEFFA3
:1001B000AC71FEFFC073FEFF2473FEFFC073FEFF31
:1001C000C073FEFF6473FEFF6D69616F750A000006
:1001D0006D69616F75320A0068756E6772790A0021
:1001E00054696D65723200004572726F7220696EDB
:1001F00020787878207461736B73200D0A000000FA
:10020000436865636B54696D65720000536574548F
:10021000780000005365745278000000000102026B
:10022000030303030404040404040404050505058E
:10023000050505050505050505050505060606066A
:10024000060606060606060606060606060606064E
:10025000060606060606060606060606070707073A
:10026000070707070707070707070707070707071E
:10027000070707070707070707070707070707070E
:1002800007070707070707070707070707070707FE
:1002900007070707070707070707070708080808EA
:1002A00008080808080808080808080808080808CE
:1002B00008080808080808080808080808080808BE
:1002C00008080808080808080808080808080808AE
:1002D000080808080808080808080808080808089E
:1002E000080808080808080808080808080808088E
:1002F000080808080808080808080808080808087E
:10030000080808080808080808080808080808086D
:0C03100008080808080808080808080881
:10031C001000000000000000017A5200017C010175
:10032C001B0D02004C000000180000008882FEFF2C
:10033C00DC05000000440E307089039507810188AC
:10034C000292049305940696089709980A990B9AB9
:10035C000C0370020AC144C844C944D244D344D4E7
:10036C0044D544D644D744D844D944DA440E004446
:10037C000B00000050000000680000001488FEFF15
:10038C000005000000440E507488028903930599FF
:10039C000B810192049406950796089709980A9A7E
:1003AC000C9B0D0320010AC144C844C944D244D358
:1003BC0044D444D544D644D744D844D944DA44DB55
:0803CC00440E00440B00000088
:1003E000AAAAAAAA08000000FC8F010009000000C8
:0C03F00001000000FFFF0000FFFF000004
:040000058000004037
:00000001FF
